:10000000004000203D6500007D6500007F65000028
:1000100000000000000000000000000000000000E0
:1000200000000000000000000000000081650000EA
:1000300000000000000000008365000085650000EE
:1000400087650000E93A00006169000087650000EB
:1000500087650000000000008765000087650000DC
:1000600087650000396C0000876500008765000027
:1000700087650000876500008765000087650000D0
:10008000876500009D6D00008765000087650000A2
:1000900087650000876500008765000087650000B0
:1000A0008765000087650000000000000000000078
:1000B0000000000000000000000000000000000040
:1000C000054B0648033310B51B1A062B03D9044B06
:1000D000002B00D0984710BDAC020020AC020020DD
:1000E000000000000648074910B5091A8910CB0F17
:1000F0005918491003D0044B002B00D0984710BD6D
:10010000AC020020AC0200200000000010B5074C3B
:100110002378002B09D1FFF7D3FF054B002B02D02A
:10012000044800E000BF0123237010BDAC02002092
:100130000000000068B10000094B10B5002B03D08F
:100140000849094800E000BF08480368002B02D1B5
:10015000FFF7C8FF10BD064B002BF9D09847F7E713
:1001600000000000B002002068B10000A8020020DA
:1001700000000000164B002B00D1144B9D4640227E
:1001800092029A1A924600218B460F461348144A4F
:10019000121A08F0E2FC0F4B002B00D098470E4BD0
:1001A000002B00D098470020002104000D000D48CE
:1001B000002802D00C4800E000BF08F08BFC2000B3
:1001C000290006F0E5FB08F05FFCC04600000800CF
:1001D000004000200000000000000000AC020020F1
:1001E00080260020000000000000000001230340E2
:1001F0000200181E04D1042A03D91068000900E087
:100200000020704710B50400FFF7F0FF0300002046
:1002100083420BD0013B9B00181DE2181279002A83
:1002200003D001338342F8D100E0180010BD012251
:10023000096810B5114201D0002903DA102000F03E
:1002400083F903E04910062002F09CF810BD09680C
:1002500010B5CB0701D5002903DA102000F074F99E
:1002600006E04910033189100022052002F08AF8C7
:1002700010BD70B50D68AB0728D1042D26D90F230A
:100280002A684E681340062B09D12800FFF7AEFFFD
:10029000012383421DDC9A00AE500133F9E7052BA0
:1002A00014D1F30703D4132000F04EF912E07610B6
:1002B000FF2EF8D82800FFF799FF2C1D230080009F
:1002C0002018984205D91E700133FAE70B2000F080
:1002D0003BF9002070BD70B50C681120E3072DD5E7
:1002E0004D68AB0729D1042D27D90F262B68641040
:1002F0001E40062E0BD1002C04DD2800FFF776FFF0
:10030000844201DD122019E0A400605918E0331F77
:10031000012B12D82800FFF769FF8000042E02D1BC
:100320002800FFF76FFF002CECDDA042EADB012381
:100330002C19E0784000184302E00B2000F004F98B
:1003400070BDF8B501230C6811201C422FD0032585
:100350004E6835402AD1042E28D90F233268641004
:100360008F681340062B0BD1002C04DD3000FFF703
:100370003DFF844201DD122019E0A400A75113E0E3
:10038000052B13D1002CF6DD3000FFF72FFF800086
:100390008442F0DC01231F4201D1132007E07F10CB
:1003A000FF2FFAD83419E770280002E00B2000F084
:1003B000CBF8F8BD086810B5830717D1042815D904
:1003C0000F2302681340062B02D1FFF70FFF0BE04B
:1003D000052B05D1FFF70AFFC0000123184308E0F1
:1003E000042B03D1FFF70EFF4000F6E70B2000F0CF
:1003F000ABF810BD012303400200181E01D05010BD
:1004000002E00D22014B1A707047C046C80200205E
:10041000012303400200181E04D1042A03D91068E6
:10042000000900E00020704770B50D000400FFF7E0
:10043000EFFF86002800FFF7EBFF830000209E42BD
:100440000ED1231D9E1904351A009E4207D9297822
:100450001278013301358A42F6D0002000E00120F5
:1004600070BD0000F0B585B00393019002912D4E50
:100470002D4B002A02D002223270013A00251A6068
:100480001B68F554019B9D424ADA029AAB00D05892
:10049000254B1C68C8239B0037191C1B01231842DD
:1004A00002D04310214A1FE0214A002802D004282C
:1004B00005D1204A2100380008F016FF18E0042872
:1004C00010D90F2302681340042B04D101F096FFCA
:1004D000194A030008E0062B05D1FFF799FF174AD8
:1004E000030001E00123164A2100380008F0FCFE59
:1004F000300008F05FFF039B0B4A002B01D1106016
:100500000CE0019B013B9D42F9DA0E4B9842F6DC70
:10051000431C1360202232540022F2540135B1E70B
:1005200005B0F0BDD4020020D0020020D9A0000008
:10053000ACA00000B2A00000CAAA0000B7A0000052
:10054000C8A000001F030000014B18700020704776
:10055000C802002070B501F071FD094C0100251D95
:100560001F22280008F02DFF280008F023FF042395
:1005700004308008000118432060200070BDC04690
:10058000F4050020C368F0B59D00836889B05D194B
:10059000030018330693036903909E00069B9F197E
:1005A00043699E000193069B9E19D54B1B78002B37
:1005B0000FD17F222B68D3491C1213409B005B583C
:1005C00001960435029235E0CD4B1B78002B29D0E3
:1005D000019E039BCA4C9B6821780193EA1A039BF6
:1005E00092109B7812021A43039B587803F062FE24
:1005F0000023039A2370137001960497039B069AB5
:100600009B68ED1A0293039BAD10DD60049B9F1A5B
:10061000039BBF101F61019B9B1A039A9B105361A0
:1006200001F086FC2B68029A1C121340B54A9B000D
:100630009B5804359F46039B587803F033FE0023F4
:10064000039A1370D9E7069B3A1DD11AAC4BDB29EC
:1006500003DD1A22019E1A70BBE71B783C60002B59
:1006600002D0019E1700B4E72B6802991C120B40C0
:10067000A4499B005B5817000435DBE7069B3A1D35
:10068000D11A9F4BDB2903DD1A22019E1A70A0E7C5
:1006900028681B78291D3860002B03D0019E1700A5
:1006A0000D0096E76B6802991C120B4095499B0060
:1006B0005B5817000835BDE7069B3A1DD11A904BD1
:1006C000DB2903DD1A22019E1A7082E7A4001B7841
:1006D0002C193C60002B02D0019E170079E72B6893
:1006E00002991C120B4087499B005B581700043588
:1006F000A0E7069B3A1DD11A814BDB2903DD1A22A4
:10070000019E1A7065E78048A40021581B78396063
:10071000002B02D0019E17005BE72B6802991C1288
:100720000B4078499B005B581700043582E7043F73
:10073000754B3A68A400E250714B1B78002B01D036
:10074000019E46E72B68029A1C1213406D4A9B00DB
:100750009B5804356EE76C4BA600F058FFF74AFE35
:10076000043F04003868FFF745FE24180120664B5B
:1007700064000443F450624B1B78002B01D0019EAF
:1007800027E72B68029A1C1213405E4A9B009B5875
:1007900004354FE7069B3A1DD11A594BDB2903DD7F
:1007A0001A22019E1A7014E70198069C0121A042AA
:1007B00002D901000C3909681B783960002B02D07E
:1007C000019E170005E72B6802991C120B404D494A
:1007D0009B005B58170004352CE7069B3A1DD11A85
:1007E000474BDB2903DD1A22019E1A70F1E60199BD
:1007F000069881420AD90B000C3B1B6843495B10E9
:100800006418E41A019BA400E35802E0182119704F
:1008100000233B603A4B1B78002B02D0019E17004F
:10082000D7E62B6802991C120B4036499B005B5897
:1008300017000435FEE6019B069A93420CD90C3B47
:100840001968324B3E1FE3184910591A3268019B50
:100850008900CA50370002E01822294B1A70284B31
:100860001B78002B01D0019EB3E62B68029A1C1264
:100870001340244A9B009B580435DBE6019B069AF3
:10088000934220D9214B3E1FE318019C04930C3C5A
:100890002368049A5B10D31A019A9B009858FFF7BB
:1008A000A9FD07903068FFF7A5FD2468049B64103C
:1008B0001C1B079BA4001F1801207F00019B0743FE
:1008C000E750370002E018220D4B1A700C4B1B78D2
:1008D000002B01D0019E7CE62B68029A1C1213406B
:1008E000084A9B009B580435A4E6069B3A1DD11A82
:1008F000034BDB290CDD1A22019E1A7069E6C04603
:10090000C8020020ECA00000C4230020FDFFFF3F30
:100910000199A40061581B783960002B02D0019E18
:10092000170056E62B6802991C120B40D0499B0019
:100930005B58170004357DE6043F019B3A68A4002C
:10094000E250CC4B1B78002B01D0019E41E62B6876
:10095000029A1C121340C64A9B009B58043569E654
:10096000019BA4001C192368043F38685E10FFF740
:1009700041FD36180120BF4B76001B7806432660E8
:10098000002B01D0019E24E62B68029A1C12134012
:10099000B74A9B009B5804354CE6069BA4003F1BBE
:1009A000B44CBB420DD82378002B01D0019E10E639
:1009B0002B68029A1C121340AD4A9B009B580435C9
:1009C00038E6AD4801F08EFC2378002B01D0019E63
:1009D000FFE52B68029A1C121340A54A9B009B5806
:1009E000043527E6A300ED18002C00DA05E6A14B3C
:1009F0001B78002B01D0019EEBE52B68029A1C129C
:100A000013409B4A9B009B58043513E63B1F0493FD
:100A10001B680793042B04D1A300ED18002C00DA07
:100A2000ECE5944B1B78002B02D0019E049FD0E58F
:100A30002B68029A1C1213408D4A9B009B58049FFE
:100A40000435F7E53B1F04931B68042B06D0A20076
:100A5000AD18002C02DA002B00D1CFE5854B1B78B6
:100A6000002B02D0019E049FB3E52B68029A1C1252
:100A700013407F4A9B009B58049F0435DAE53A1FD8
:100A800013685B10013B002B07DD01215B00A40014
:100A90000B4304972D191360B0E5764B17001B78B4
:100AA000002B01D0019E94E52B68029A1C12134082
:100AB0006F4A9B009B580435BCE53A00069B0C32FC
:100AC000D31ADB2B04DD1A226A4B019E1A7080E5D3
:100AD000FF2361005B000B4001210B433B60039B44
:100AE00006989B6824120493ED1A039BAD109B7823
:100AF0002D021D43019B8D401B1A9B108B400B4305
:100B0000BB60039B0D437D609C70E4B25B4BE400D3
:100B10000399E35816008B6056490978002903D0E1
:100B200008331D00170054E51D0002999B680C3521
:100B30001C120B404E499B005B580192170079E54F
:100B40003B1F1C68069A019B93422AD104970A20F6
:100B5000E30716D4A3070DD1042C0BD90F23226869
:100B60001340042B06D1200001F048FC08F022FCC1
:100B7000063006E00720042C03D0002C01D0802092
:100B80008000643003F03CF9002801D1043D35E5D4
:100B9000039B2100587803F09FFB0023039A1370F6
:100BA0002CE5019B019A0C3B1B6803995B109B0091
:100BB0005B421E00D3180C3B1C601300083B1B68F3
:100BC000083E97195A108A70D2B22C49D2005B00A5
:100BD00055589B0A039A9B009560ED18019B043BB6
:100BE0001E68069B7610B6009E19224B1B78002BC0
:100BF00000D0EEE42B68029A1C1213401C4A9B00A2
:100C00009B580196043515E53B1F1868FFF7F2FB6A
:100C1000A40006003F1B1E2834DC00280EDC154B08
:100C20001B78002B01D0019ED3E42B68029A1C1282
:100C300013400F4A9B009B580435FBE401F0E4F994
:100C4000033E361801F0E0F90D4B801B9842F9D8AD
:100C5000084B1B78002B01D0019EBAE42B68029A46
:100C60001C121340024A9B009B580435E2E4C04624
:100C7000ECA00000C8020020DCA00000CC1B00207B
:100C80009F8601000123039A137001F0BDF9039BB5
:100C90000A3886195E60B0E43B1F1868FFF7AAFBAC
:100CA000A40004903F1B00280EDCCA4B1B78002BCD
:100CB00001D0019E8DE42B68029A1C121340C64A93
:100CC0009B009B580435B5E4C44B049A019E9A429C
:100CD00003DD1D22BF4B1A707BE40123039A1370BE
:100CE00001F092F9FA23049A9B005343039A0A3BBA
:100CF0001B18536081E4A300FF1A002320001A0090
:100D00003900FFF7AFFBB64EB64C3168200003F058
:100D100033FA3168200003F0E6FA3168200001F070
:100D200043FCAC4B1B78002B01D0019E51E42B6897
:100D3000029A1C121340A84A9B009B58043579E480
:100D4000A44BA4001B783F1B002B01D0019E40E464
:100D50002B68029A1C1213409F4A9B009B58043533
:100D600068E403F093F801F0E3F83B1F18680028EB
:100D700023D1083B1868C30701D5401016E083074C
:100D80000FD104280DD90F2302681340062B02D17E
:100D9000FFF73EFB0AE0052B03D1FFF739FB80008C
:100DA00004E019228B4B019E1A7012E43A000121D3
:100DB0004300083A0B43136001E04010013800285B
:100DC00032DD012243001343391F0B603B00083B17
:100DD0001B681341181A3B000C3B1B68134203D0DD
:100DE0008018A400904015E0990717D1042B15D95D
:100DF0000F211E683140062906D101308000C358FA
:100E0000019AA400A35010E0052907D11818007911
:100E1000A4004000019B1043E05006E019226D4BF6
:100E2000019E1A70FFF7D5FB04356A4B1B78002B27
:100E300002D0019EFFF7CDFB2B68029A1C121340D3
:100E4000654A9B009B580435FFF7F4FBA300069A04
:100E5000FB189B1ADB2B01DC012205E01A225D4BFB
:100E6000019E1A70FFF7B5FB631E002C03DD3A608C
:100E70001C000437F8E7574B1B78002B02D0019E6B
:100E8000FFF7A7FB2B68029A1C121340524A9B00E3
:100E90009B580435FFF7CEFB069A3B1D9B1A4D4E1F
:100EA000DB2B04DD1A233370019EFFF792FB019BBD
:100EB000069AA400934218D93B1F1868FFF79AFAC4
:100EC000002810DD019B0C3B1B685B1098420ADC7C
:100ED0009A07D31A1818444BC018019B8000C258B7
:100EE0003B1B1A6003E0202300E018233370394BCA
:100EF0003E1B1B78371D002B02D0019EFFF769FBBC
:100F00002B68029A1C121340334A9B009B580435ED
:100F1000FFF790FBA3009C46F81A002C04DC1C226F
:100F20002C4B00261A7015E0002103685B10012687
:100F30008A008258164003D10D22264B1A7009E010
:100F40005210934200DD130001318C42EFDC012688
:100F50005B001E4363460660FE1A1E4B371D1B785E
:100F6000002B02D0019EFFF734FB2B68029A1C1263
:100F70001340194A9B009B580435FFF75BFBA30005
:100F80009C46F81A002C04DC1C22124B00261A7016
:100F900015E0002103685B1001268A008258164084
:100FA00003D10D220B4B1A7009E05210934200DA64
:100FB000130001318C42EFDC01265B001E436346C7
:100FC0000660FE1A034B371D1B78002B0ED0019EC6
:100FD000FFF7FFFAC8020020ECA0000080EE360008
:100FE000D0020020D4020020FCFFFF3F2B68029AB1
:100FF0001C121340D84A9B009B580435FFF71AFB7C
:101000003B00083B1868FFF7F5F93B1F0490186890
:10101000FFF7F0F9049AA600BC1B0023824200DA15
:1010200004332360CD4BBE1B1B78371D002B02D031
:10103000019EFFF7CEFA2B68029A1C121340C64A93
:101040009B009B580435FFF7F5FAA300FE1A0493A2
:101050003B00083B1868FFF7CDF93B1F04001868F8
:10106000FFF7C8F9E20FC317A04253419B0033605A
:10107000049BFE1AB94B371D1B78002B02D0019E32
:10108000FFF7A7FA2B68029A1C121340B24A9B0082
:101090009B580435FFF7CEFA3B00083B18683B1F0E
:1010A0001968A300884202D1FB1A042222E0042816
:1010B0001ED90122104201D0114219D1032630421B
:1010C00015D10F2302681A40042A10D131420ED1E3
:1010D00004290CD90A681340042B08D1FFF7A4F99E
:1010E000431E9841A600BE1B8000306003E0A300B1
:1010F0000022FB1A1A60994BA4001B783E1B371D77
:10110000002B02D0019EFFF764FA2B68029A1C1292
:101110001340914A9B009B580435FFF78BFA3B0024
:10112000083B18683B1F1968A300884202D1FB1ACC
:10113000002223E004281FD90122104201D01142CD
:101140001AD10326304216D10F2302681A40042A0E
:1011500011D131420FD104290DD90A681340042B53
:1011600009D1FFF761F9030058425841A600BE1BA0
:101170008000306003E0A3000422FB1A1A60774B62
:10118000A4001B783E1B371D002B02D0019EFFF7E9
:1011900020FA2B68029A1C1213406F4A9B009B583E
:1011A0000435FFF747FAA300FE1A04933B00083BFF
:1011B0001868FFF71FF93B1F04001868FFF71AF9BA
:1011C000E217C30F844253419B003360049BFE1A15
:1011D000624B371D1B78002B02D0019EFFF7F9F9F7
:1011E0002B68029A1C1213405B4A9B009B580435E3
:1011F000FFF720FA3B00083B1868FFF7FBF83B1F9E
:1012000004901868FFF7F6F8049AA600BC1B0023A8
:10121000824200DD04332360504BBE1B1B78371D18
:10122000002B02D0019EFFF7D4F92B68029A1C1202
:101230001340494A9B009B580435FFF7FBF93B1FBD
:101240001B68A400043B591E8B413A1B9B00136092
:10125000424B171D1B78002B02D0019EFFF7B9F9F6
:101260002B68029A1C1213403B4A9B009B58043582
:10127000FFF7E0F9A300FC1A04933B00083B186851
:10128000FFF7B8F83B1F06001868FFF7B3F83618E9
:101290000120049B760006432660FE1A2F4B371D63
:1012A0001B78002B02D0019EFFF793F92B68029A5E
:1012B0001C121340284A9B009B580435FFF7BAF9CB
:1012C000A300FE1A04933B00083B1868FFF792F84E
:1012D0003B1F04001868FFF78DF8241A0120049BB7
:1012E000640004433460FE1A1C4B371D1B78002B2E
:1012F00002D0019EFFF76DF92B68029A1C12134071
:10130000154A9B009B580435FFF794F9A300FC1A7B
:1013100004933B00083B1868FFF76CF83B1F06007E
:101320001868FFF767F846430120049B76000643E0
:101330002660FE1A094B371D1B78002B02D0019E38
:10134000FFF747F92B68029A1C121340024A9B00D0
:101350009B580435FFF76EF9ECA00000C80200208E
:101360003B1F1868FFF746F8A30006000493FC1A19
:10137000002803D11F22E84B1A700AE03B00083B0B
:101380001868FFF737F8310005F0ACFD0126400082
:101390000643049B2660FE1ADF4B371D1B78002B8B
:1013A00002D0019EFFF715F92B68029A1C12134018
:1013B000DA4A9B009B580435FFF73CF93B1F18683D
:1013C000FFF718F8A30006000493FC1A002803D1C5
:1013D0001F22D14B1A700AE03B00083B1868FFF748
:1013E00009F8310005F064FE012649000E43049B14
:1013F0002660FE1AC84B371D1B78002B02D0019EB9
:10140000FFF7E7F82B68029A1C121340C34A9B00AF
:101410009B580435FFF70EF93B1F1868FEF7EAFFEB
:10142000C317C0185840012340001843BA4BA4000A
:101430001B783E1B3060371D002B02D0019EFFF74A
:10144000C8F82B68029A1C121340B44A9B009B58A0
:101450000435FFF7EFF8A300FE1A07933068012C5C
:1014600003D1FEF7C7FF049008E0FEF7C3FF0400B6
:101470007068FEF7BFFF0130031B0493049B002B31
:1014800001DC0123049307F0E1FE049905F010FE4E
:101490000C190121079B64000C433460FE1A9E4B1B
:1014A000371D1B78002B02D0019EFFF792F82B68A6
:1014B000029A1C121340994A9B009B580435FFF76F
:1014C000B9F8A300FE1A31002000049300F0A8FF31
:1014D000049B3060FE1A904B371D1B78002B02D006
:1014E000019EFFF776F82B68029A1C1213408B4A74
:1014F0009B009B580435FFF79DF8A300FE1A049348
:101500003B00083B1868FEF775FF3B1F0400186896
:10151000FEF770FF04400120049B64000443346024
:10152000FE1A7D4B371D1B78002B02D0019EFFF762
:1015300050F82B68029A1C121340784A9B009B5863
:101540000435FFF777F8A300FC1A04933B00083B2F
:101550001868FEF74FFF3B1F06001868FEF74AFFAA
:1015600006430120049B760006432660FE1A6A4B60
:10157000371D1B78002B02D0019EFFF72AF82B683D
:10158000029A1C121340654A9B009B580435FFF7D2
:1015900051F8A300FC1A04933B00083B1868FEF7BF
:1015A00029FF3B1F06001868FEF724FF4640012074
:1015B000049B760006432660FE1A574B371D1B78A6
:1015C000002B02D0019EFFF704F82B68029A1C1230
:1015D0001340524A9B009B580435FFF72BF83B1FE2
:1015E0001868FEF707FFC0430123400018434A4B29
:1015F000A4001B783E1B3060371D002B02D0019EDB
:10160000FEF7E7FF2B68029A1C121340434A9B0027
:101610009B580435FFF70EF8A300FE1A04933B0015
:10162000083B1868FEF7E6FE3B1F04001868FEF74B
:10163000E1FE8440012364001C43049B3460FE1AD5
:10164000354B371D1B78002B02D0019EFEF7C1FFE2
:101650002B68029A1C121340304A9B009B58043599
:10166000FEF7E8FFA300FE1A04933B00083B18684E
:10167000FEF7C0FE3B1F04001868FEF7BBFE0441E6
:10168000012364001C43049B3460FE1A224B371D67
:101690001B78002B02D0019EFEF79BFF2B68029A5D
:1016A0001C1213401D4A9B009B580435FEF7C2FFD5
:1016B0003B000C3B1868FEF79DFE3B00083B060014
:1016C0001868FEF797FEF1170200C317300005F007
:1016D00041FD3B1F049005911868FEF78BFE020048
:1016E0000498059905F0EAFC0123400018430A4BD1
:1016F000A4001B783E1B3060371D002B02D0019EDA
:10170000FEF767FF2B68029A1C121340034A9B00E6
:101710009B580435FEF78EFFC8020020ECA00000A5
:10172000A300FE1A310020000493FEF780FD049B05
:101730003060FE1AE54B371D1B78002B02D0019E4E
:10174000FEF747FF2B68029A1C121340E04A9B00E9
:101750009B580435FEF76EFFA300FE1A31002000EF
:101760000493FEF774FD049B3060FE1AD74B371DBF
:101770001B78002B02D0019EFEF72BFF2B68029AEC
:101780001C121340D24A9B009B580435FEF752FFAF
:10179000A300FF1A39002000FEF76BFDCB4B1B782E
:1017A000002B02D0019EFEF714FF2B68029A1C1238
:1017B0001340C74A9B009B580435FEF73BFFA3002C
:1017C000FE1A310020000493FEF785FD049B306073
:1017D000FE1ABE4B371D1B78002B02D0019EFEF770
:1017E000F8FE2B68029A1C121340B94A9B009B58C2
:1017F0000435FEF71FFFA300FF1A39002000FEF793
:10180000A0FDB24B1B78002B02D0019EFEF7E1FE3B
:101810002B68029A1C121340AD4A9B009B5804355A
:10182000FEF708FFA300FE1A310020000493FEF724
:10183000C1FD049B3060FE1AA44B371D1B78002BA2
:1018400002D0019EFEF7C5FE2B68029A1C121340BF
:101850009F4A9B009B580435FEF7ECFE069A3B1D01
:1018600004939A4C9B1ADB2B04DD1A23019E2370F0
:10187000FEF7AFFE00F0D2FB0123400018432378AF
:101880003860002B03D0019E049FFEF7A2FE2B6858
:10189000029A1C1213408E4A9B009B58049F0435E9
:1018A000FEF7C8FE069A3B1D0493884C9B1ADB2B5F
:1018B00004DD1A23019E2370FEF78BFE00F0A4FBCB
:1018C000844B400018400123184323783860002BD4
:1018D00003D0019E049FFEF77CFE2B68029A1C1227
:1018E00013407B4A9B009B58049F0435FEF7A2FEE1
:1018F000A300FB1A0493012320001A000499FEF7A9
:10190000B1FD754C2068643002F07AFA002816D0D8
:10191000039B21685A78714802F0F3FC15E0A3009C
:10192000FB1A04932000012300220499FEF79AFD7C
:10193000694C2068643002F063FA002802D1043D4B
:10194000FEF75BFE654802F075FB0123039A1370F6
:1019500000F05AFB624A2368126806335343181892
:10196000039B5860FEF74AFEFEF7F4FD574BA400B8
:101970001B783E1B3060371D002B02D0019EFEF706
:1019800028FE2B68029A1C121340514A9B009B5858
:101990000435FEF74FFEA4003E1B300000F072FB42
:1019A0004A4B30601B78371D002B02D0019EFEF79A
:1019B00010FE2B68029A1C121340454A9B009B584C
:1019C0000435FEF737FEA4003E1B300000F05CFB40
:1019D0003E4B30601B78371D002B02D0019EFEF776
:1019E000F8FD2B68029A1C121340394A9B009B5841
:1019F0000435FEF71FFEA4003E1B300000F046FB3E
:101A0000324B30601B78371D002B02D0019EFEF751
:101A1000E0FD2B68029A1C1213402D4A9B009B5834
:101A20000435FEF707FEA4003F1B380000F04CFB16
:101A3000264B1B78002B02D0019EFEF7CAFD2B68B7
:101A4000029A1C121340224A9B009B580435FEF751
:101A5000F1FDA300FE1A31002000049300F056FBB4
:101A6000049B3060FE1A194B371D1B78002B02D0E7
:101A7000019EFEF7AEFD2B68029A1C121340144A19
:101A80009B009B580435FEF7D5FDA4003F1B380092
:101A900000F076FB0D4B1B78002B02D0019EFEF769
:101AA00098FD2B68029A1C121340094A9B009B5810
:101AB0000435FEF7BFFD0121200000F049FB034B78
:101AC0001B78002B0ED0019EFEF783FDC80200207C
:101AD000ECA00000FEFFFF7FD0020020D402002017
:101AE000040000202B68029A1C121340E94A9B0054
:101AF0009B580435FEF79EFD0021200000F028FBD6
:101B0000E54B1B78002B02D0019EFEF762FD2B688F
:101B1000029A1C121340DF4A9B009B580435FEF7C3
:101B200089FDA4003E1B300000F048FBDA4B30601A
:101B30001B78371D002B02D0019EFEF74AFD2B6853
:101B4000029A1C121340D34A9B009B580435FEF79F
:101B500071FDA4003E1B300000F044FBCE4B306012
:101B60001B78371D002B02D0019EFEF732FD2B683B
:101B7000029A1C121340C74A9B009B580435FEF77B
:101B800059FDA4003F1B380000F006FBC24B1B7838
:101B9000002B02D0019EFEF71CFD2B68029A1C123E
:101BA0001340BC4A9B009B580435FEF743FDA4003C
:101BB0003F1B380002F056FEB74B1B78002B02D0BB
:101BC000019EFEF706FD2B68029A1C121340B14AD3
:101BD0009B009B580435FEF72DFDA4003E1B3000F2
:101BE00002F0D4FEAC4B30601B78371D002B02D0C6
:101BF000019EFEF7EEFC2B68029A1C121340A54AC8
:101C00009B009B580435FEF715FDA4003F1B3800D0
:101C100002F0D8FDA04B1B78002B02D0019EFEF7EE
:101C2000D8FC2B68029A1C1213409A4A9B009B58BE
:101C30000435FEF7FFFCA4003E1B300002F0D8FD87
:101C4000954B30601B78371D002B02D0019EFEF7AC
:101C5000C0FC2B68029A1C1213408E4A9B009B58B2
:101C60000435FEF7E7FCA300FF1A3900200000F05E
:101C700003FF894B1B78002B02D0019EFEF7A9FCC5
:101C80002B68029A1C121340824A9B009B58043511
:101C9000FEF7D0FCA300FF1A3900200000F0B6FDCB
:101CA0007D4B1B78002B02D0019EFEF792FC2B6827
:101CB000029A1C121340774A9B009B580435FEF78A
:101CC000B9FCA300FF1A3900200000F0AFFD724BF1
:101CD0001B78002B02D0019EFEF77BFC2B68029A3A
:101CE0001C1213406B4A9B009B580435FEF7A2FC64
:101CF000A300FF1A3900200000F0C0FD664B1B78DE
:101D0000002B02D0019EFEF764FC2B68029A1C1285
:101D10001340604A9B009B580435FEF78BFCA300E0
:101D2000FE1A31002000049302F0BAFE049B3060DA
:101D3000FE1A594B371D1B78002B02D0019EFEF76F
:101D400048FC2B68029A1C121340524A9B009B5875
:101D50000435FEF76FFCA300FE1A31002000049347
:101D600002F0A6FE049B3060FE1A4B4B371D1B7819
:101D7000002B02D0019EFEF72CFC2B68029A1C124D
:101D80001340444A9B009B580435FEF753FCA300C4
:101D9000FE1A31002000049302F092FE049B306092
:101DA000FE1A3D4B371D1B78002B02D0019EFEF71B
:101DB00010FC2B68029A1C121340364A9B009B5859
:101DC0000435FEF737FCA300FE1A3100200004930F
:101DD00002F0B0FC049B3060FE1A2F4B371D1B78BD
:101DE000002B02D0019EFEF7F4FB2B68029A1C1216
:101DF0001340284A9B009B580435FEF71BFCA300A8
:101E0000FF1A3900200000F0D5FD234B1B78002B72
:101E100002D0019EFEF7DDFB2B68029A1C121340D4
:101E20001C4A9B009B580435FEF704FCA300FF1AD4
:101E30003900200000F04AFD174B1B78002B02D020
:101E4000019EFEF7C6FB2B68029A1C121340114A32
:101E50009B009B580435FEF7EDFBA300FE1A3100F2
:101E60002000049300F01EFE049B3060FE1A0A4B13
:101E7000371D1B78002B02D0019EFEF7AAFB2B68B2
:101E8000029A1C121340034A9B009B580435FEF72C
:101E9000D1FBC046ECA00000C8020020A300FF1A3E
:101EA0003900200000F0F6FB224B1B78002B02D0FB
:101EB000019EFEF78EFB2B68029A1C1213401E4AED
:101EC0009B009B580435FEF7B5FBA300FF1A3900B1
:101ED000200001F017FF174B1B78002B02D0019E4A
:101EE000FEF777FB2B68029A1C121340124A9B00E4
:101EF0009B580435FEF79EFBA300FE1A310020001C
:101F0000049301F0FFFE049B3060FE1A094B371D5D
:101F10001B78002B02D0019EFEF75BFB2B68029A18
:101F20001C121340044A9B009B580435FEF782FBA9
:101F300009B0F0BDC8020020ECA000000023F7B5F6
:101F40005A1E0192002B07DA00F0E0FD02F04EF974
:101F500002F0FCF96423019300263000194B196844
:101F60008E4201DB019BEBE7174B1A68013291426D
:101F700000DC0022F0241A601D68144F6C43E35DFE
:101F8000002B1DD0E419022B16D0012B0ED10028F6
:101F900001D100F039F8F0226A430C4B0C499B1830
:101FA0005B68C31A8B4201D80223BB54F0235D4304
:101FB000064BEB5C022B03D12000FEF7E3FAD1E7DE
:101FC0000136CBE7CC020020000000206C1200207C
:101FD0009F86010000207047002070470020704756
:101FE0000020704701220020054B06491A61585015
:101FF0000330043158508018083158501A60704727
:1020000000800040040500000122034B1A64A8224E
:10201000D20098587047C0460080004010B5FFF7C6
:10202000F3FFFA21890004F0D3FE10BD10B50100C2
:10203000014804F03DFA10BDF4110020004870473B
:10204000F4A2000070B5054E0400335C0D008B4215
:1020500002D004F037FE355570BDC046180600208A
:1020600070B50024064D635D012B05D100212000D1
:1020700004F028FE0023635501341D2CF2D170BDFD
:10208000180600200D2070473B207047036870B58C
:102090005B100120052B12D8094A9B009C58094D62
:1020A0002B5D002B05D00021200004F00BFE002347
:1020B0002B55200004F0B0FC01234000184370BDF4
:1020C00024A300001806002070B5036845685C1062
:1020D0006D1004D40B4B9D4202DD1D0000E0002575
:1020E0001C2C0DD8084E335D012B05D0012120009A
:1020F00004F0E8FD012333552900200004F01AFD07
:1021000070BDC046FF030000180600200B6870B5C4
:102110005D101C2D16D80024012804DD4C68043CF9
:10212000624262415400094E735D9C4204D021001A
:10213000280004F0C7FD7455280004F0F7FD0423BF
:10214000012800D00023180070BDC04618060020EA
:1021500070B504000D001C280ED8084E335C012B0E
:1021600004D0012104F0AEFD0123335529002000E5
:102170004D1EA94104F0C4FD70BDC04618060020E4
:10218000436810B5191F4A424A41006811004010C7
:10219000FFF7DEFF10BD000037B56A46064B694603
:1021A00030CB30C203680220042B02D100F03EFB8A
:1021B00001E000F063FB37BDECA2000010B5084C55
:1021C0006379002B05D00021052004F07BFD00235E
:1021D0006371052004F0AAFD43425841800010BD00
:1021E0001806002010B5084CE37A002B05D000211A
:1021F0000B2004F067FD0023E3720B2004F096FD32
:1022000043425841800010BD1806002070477047B7
:1022100010B5034A0421034801F060FD10BDC0461B
:1022200008000020E0A90000E12110B5490209489A
:1022300004F01CFAFFF7D6FE0A2004F0E7FB0023A7
:10224000FF21054A995401331D2BFBD100F0B2FD4B
:1022500010BDC046F411002018060020F8B50B4E42
:10226000070030000D0004F041FA041EAC4200DD0E
:102270002C003D00EB1B9C4205DD300004F040FAD1
:1022800028700135F6E72000F8BDC046F4110020A3
:1022900010B50100014804F0F1F910BDF41100205F
:1022A00010B5054C200004F0F7F9E12120004902A7
:1022B00004F0DCF910BDC046F4110020064B0120EB
:1022C0001A68064B06491A60C82200235200C850FB
:1022D00004339342FBD170474006002038060020AB
:1022E000C423002000B59BB00200054901A807F0F7
:1022F0002DF801A801F0BAFE02F028F8FCE7C0466C
:102300003CA3000037B5184D04002868002801D010
:1023100006F010FCA400200006F002FC2860002853
:1023200001D1124809E001AB984208D2104B0219C2
:102330006B440193934202D20E48FFF7D3FF042867
:1023400002D808302860083C2B680B4A1C1913601F
:102350000A4BC8221C600120002309495200C850C2
:1023600004339342FBD137BD400600204DA300004B
:102370001CFCFFFF7DA30000380600203C06002067
:10238000C423002070B50D4D0D4E2B684C1CA400CD
:1023900036681C19B44203D90A20FEF7D5F80BE0C1
:1023A0002C601D00AC4201D904C5FBE70F220901D6
:1023B000104008431860180070BDC0463806002061
:1023C0003C0600200322CB1C70B50C00D91711402D
:1023D000C9180500891000220420FFF7D3FF00234D
:1023E000A34204DAE95CC21811710133F8E7E14352
:1023F0000023C917214041180B7170BD10B5830728
:1024000006D1042804D90F2304C81340042B03D099
:102410000E20FEF799F8014810BDC04616A900002D
:1024200010B503240868044006D1042804D90F23FA
:1024300002681340042B01D00E2011E0FFF7DEFFED
:102440000378233B5942594110224018210007F0DC
:102450005DF880239B05C218054B9A4203D91420CE
:10246000FEF772F802E001234000184310BDC04699
:10247000FFFFFF3F70B501240B680D001C4001D029
:102480005C1002E00D20FEF75FF8200004F0A2FFD0
:10249000264904F08BFE06F065FA02F077FE002272
:1024A000234B05F019FC0023002204F049FE01240F
:1024B0002B681C40002819D0002C01D05C1002E0D1
:1024C0000D20FEF741F8200004F084FF174904F0C6
:1024D0006DFE06F047FA02F059FE0022144B05F09B
:1024E000FBFB0022134B04F0BDFF18E0002C01D0D1
:1024F0005C1002E00D20FEF727F8200004F06AFFD0
:102500000A4904F053FE06F02DFA02F03FFE0022C5
:10251000074B05F0E1FB0022064B05F057FE06F0E5
:10252000A9F901234000184370BDC046D3023739D2
:102530000000D0400000E03F10B5034A02210348EC
:1025400001F0CCFB10BDC04628000020E8A300002D
:102550000020704710B51E20FDF7F6FF10BD10B526
:102560001E20FDF7F1FF10BD10B51E20FDF7ECFF9A
:10257000002010BD10B51E20FDF7E6FF002010BDA5
:1025800010B51E20FDF7E0FF10BD10B51E20FDF7B1
:10259000DBFF10BD10B51E20FDF7D6FF10BD10B536
:1025A0001E20FDF7D1FF10BD7047000010B5034A93
:1025B0000921034801F092FB10BDC04638000020FD
:1025C000FAA300000123034A1360034A10689840ED
:1025D000184370474C06002054060020202800D9DC
:1025E0000020084B8000C25801239340064A074947
:1025F0001360074A1160074A07491160074A1360D0
:102600007047C04670AC0000480600200805005026
:10261000640600205C0600200C05005018050050E0
:10262000F0B5EFF310810123194083F31088134EA6
:10263000134AB4461268013A9340124A1468124A87
:102640001568124A002B15D0166803420BD026607D
:10265000C046C046C046C046C046C046C046C0464A
:1026600016682E6004E067463E601668084F3E60BC
:102670005B08E7E781F31088F0BDC046080500500D
:10268000C8000020640600205C06002048060020E8
:102690000C0500500B6810B50200D80701D5581082
:1026A00001E0012040421823012A03DD4A68042A80
:1026B00000D10833024A1360FFF790FF002010BDDD
:1026C000C800002030B585B001AD0C2206492800B5
:1026D00006F03AFA0024285D01210134FFF7B2FC2C
:1026E0000C2CF8D105B030BD86A40000F0B53B4CF1
:1026F00085B0210003220C31684606F025FA21003E
:1027000009220F3101A806F01FFAFFF787FC344BAE
:10271000344CC0182368984201D2002323602568F6
:10272000002D3ED12E006B4604339F5D0121380001
:10273000FFF788FC01360121380004F0E1FA092E88
:10274000F1D100266B469F5D01213800FFF77AFC2E
:1027500001360021380004F0D3FA032EF2D1C8204C
:1027600080000138C046C046C046C046C046C0468C
:10277000C046C046C046C046C046C046F1D1002152
:102780000420FFF75FFC00266B460021985D0136B0
:10279000FFF758FC032EF7D1FFF740FC1330206001
:1027A00019E0FFF73BFC23680025984213D304206F
:1027B00004F032F90C4B0D4EC01801D4306000E02B
:1027C00035603068032104F08DFB00230125084AA1
:1027D000306023601360280005B0F0BD86A40000BF
:1027E0001027000044060020C8FEFFFF540600200A
:1027F0004C06002010B50124044001D0441002E032
:102800000D20FDF7A1FE200010BD00000022054BA9
:1028100010B51A60044B1B68934201D002F0B2F964
:10282000002010BD580600201811002070B508685F
:102830000D00FFF7DFFF04006868FFF7DBFF631E92
:102840000100042B14D8451E042D11D805226A431B
:10285000D318012215009D402B00064805682B4324
:102860000360054B1B68002B02D0200002F08BF99F
:10287000002070BD580600201811002070B50868AF
:102880000D00FFF7B7FF04006868FFF7B3FF631E92
:102890000100042B14D8451E042D11D805226A43CB
:1028A000D31801229A401300064802689A43064B47
:1028B00002601B68002B03D00022200002F063F9A5
:1028C000002070BD5806002018110020F0B505004A
:1028D00085B008680C00FFF78DFF0390022D08DD1E
:1028E0006068FFF787FF0700A068FFF783FF040019
:1028F00001E00124270005236343053B02930123E4
:1029000026000193231D9E4234DC3D003B1D9D4269
:102910002BDC731E042B23D86B1E042B20D8029BA8
:10292000039A591E019B49191A40204B0AD00122D3
:102930008A4019680A431A601D4B01221B68002B4C
:102940000ED009E001208840010018688843186013
:10295000174B1B68002B03D03100280002F013F93D
:10296000019B01355B000193D0E7029B01360533E3
:102970000293C7E73D1D042D15D8012C13D1260065
:102980003300AB40094A11689943094B11601B6839
:10299000002B04D0781D0022210002F0F4F801344D
:1029A0000535062CECD1002005B0F0BD58060020FE
:1029B000181100202D4BF7B51B680C00002B03D11C
:1029C00001204042FFF70AFE01262468344219D054
:1029D000FF226310180212041040FF22611212023B
:1029E0000A40DBB210431843214B1B68202B06D151
:1029F000B440204BA40EA400E35800021843FFF794
:102A00000FFE30E0032525402DD1042C2BD90F23B8
:102A100022681340062B26D1FF27130901933F0498
:102A2000019B9D421FDAAB00E3185A68324218D06E
:102A3000531018023840FF21844609025012084002
:102A40006146DBB208431843094B1B68202B06D1B3
:102A50005200920E074B9200D35800021843FFF722
:102A6000DFFD0135DCE70020FEBDC0464806002042
:102A7000C800002014A50000086810B5C30703D5DE
:102A8000FFF7B8FE054B1860054B1B68002B03D001
:102A9000024B186802F078F8002010BD580600209C
:102AA000181100200868F8B5C30702D5FFF7A2FE89
:102AB0000BE0830726D1042824D90F2203681A408B
:102AC000042A1FD11B091DD000790300203B5E2B77
:102AD00018D80522002053430B4E9D18043AAB42F0
:102AE0000CD0052110249F5D3C4200D08018013994
:102AF000520064100029F7D10133F0E701234000B0
:102B0000184300E00120F8BD14A600007FB5A44ED4
:102B10003368002B0BD1A34A1268002A07D1A24BBD
:102B20001B68002B00D139E1FFF7E0FD36E19F4D36
:102B30002A68002A2AD19C4A1268002A07D0FFF787
:102B4000D5FD002800D129E1FFF7BCFD05E0954A3D
:102B50001268002A01D1002BF6D1924B19681A0095
:102B6000002911D03468002C0ED101AD0C229049FF
:102B700028001C6005F0E8FF285D00210134FFF704
:102B800061FA0C2CF8D109E13368136000211A2096
:102B900004F0B6F800211B2004F0B2F800211C203C
:102BA00004F0AEF82E68012E56D0022E00D19CE023
:102BB000002E00D0ECE0013631007A4C032023686F
:102BC000994304F09DF80420216801400B0059420C
:102BD000594104F095F8102123680A200B4059420E
:102BE000594104F08DF88021236809010B405942B6
:102BF0005941062004F084F88021236809020B4023
:102C000059425941072004F07BF88021236849028A
:102C10000B4059425941092004F072F88021236881
:102C200089020B4059425941192004F069F880216A
:102C30002368C9020B4059425941182004F060F83A
:102C4000802321681B030B4059425941172004F08F
:102C500057F831001A2099E00221524C17202368BE
:102C60000B405942594104F04BF8082123681820C1
:102C70000B405942594104F043F880212368C900B0
:102C80000B4059425941042004F03AF8802123684E
:102C900049010B40594259410A2004F031F8802182
:102CA0002368C9010B4059425941032004F028F818
:102CB0008021236889030B4059425941092004F0BF
:102CC0001FF8802321681B040B40594259411920E9
:102CD00004F016F83100062004F012F83100072045
:102CE00004F00EF831001B2050E020212D4C17205D
:102CF00023680B405942594104F002F840212368EF
:102D000018200B405942594103F0FAFF80212368F3
:102D100019200B405942594103F0F2FF80212368EA
:102D200049000B4059425941092003F0E9FF802135
:102D3000236889000B4059425941072003F0E0FF06
:102D40008021236889010B4059425941062003F034
:102D5000D7FF8021236849030B40594259410A207B
:102D600003F0CEFF80212368C9030B40594259412B
:102D7000032003F0C5FF802321685B040B40594208
:102D80005941042003F0BCFF01211C2003F0B8FFCF
:102D90002B680321581C04F08BF929607FBDC046C5
:102DA00058060020500600204C0600206006002037
:102DB00086A40000012010B54042FFF70FFC10BDB3
:102DC00010B5034A0921034800F088FF10BDC04632
:102DD000800000209EA4000030B502248025094B0D
:102DE000094AED009C505C59002CFCD0A124E40061
:102DF000884204D28025ED0018514019F8E70021DF
:102E0000995030BD00E001400405000010B50028D5
:102E100004D19820A6214002890203E0A620802147
:102E20008002C902FFF7D8FF10BD002802D0A623F8
:102E30009B0201E098235B021B6800201A0E532AB4
:102E400001D11B02180A704730B501248025064ABB
:102E5000064BED00D4505459002CFCD001600021E9
:102E6000014AD15030BDC04600E0014004050000D9
:102E700010B5002802D0A620800201E09820400270
:102E8000A6230902DB05090A1943FFF7DDFF10BD80
:102E9000F0B50124802503000F4F08000F49ED0015
:102EA0007C507C59002CFCD09C46002810DD5478C6
:102EB00016789378240234431B0423431C00D378F0
:102EC00001381B062343644608C40432A446ECE7D9
:102ED00000237B50F0BDC04600E001400405000027
:102EE00070B505004B680A009C1C2100FFF7D0FF5D
:102EF000A000281870BD0000154B1B68002B04D0E3
:102F00008021A623C9029B0203E0A62198238902FF
:102F10005B02002807D1191D5B6802001B0E522BB3
:102F200014D10A0012E0002281420FD903681B0E5F
:102F3000522B0BD1436802339B00C318994205D929
:102F40001A68110E0022522900D11A001000704791
:102F50006808002070B50020FFF7CEFFFF260500AF
:102F6000002808D003681C143440FFF7C5FFDA2C92
:102F7000F6D10500F4E7280070BD00008022F0B50E
:102F80005200A1B00021654805F0E7FD8022002134
:102F90005200634805F0E1FD624C23681A00039378
:102FA00053425A4110000492FFF730FF039B0594EF
:102FB000002B01D15C4C00E05C4C0020FFF7CAFF05
:102FC000FF270500002D7CD02A68131412123A4006
:102FD0003B4002921A000A3A092A42D84F4B029A01
:102FE000995C002968D11022514805F0B6FD2E00E9
:102FF000336802991A123A40914217D11A143A4092
:103000000B2A06D0132A0CD00A2A0FD1484B1E6077
:103010000CE03B40022B09DC454A9B00D3185E6064
:1030200004E010220021424805F097FD3000FFF730
:1030300063FF061EDCD13E4B196800290FD020002B
:10304000FFF74EFF04003B4E3168002903D02000FB
:10305000FFF746FF0400384B0436B342F4D12F4B40
:1030600027E01A00153A082A26D82D4A0299565CFC
:10307000002E21D1152B00D12E00280003681A1430
:103080003A40152A03D01D2A07D1002605E0029AEE
:103090001B123B409A4200D10600FFF72DFF00288B
:1030A000ECD1002E04D020003100FFF719FF0400FE
:1030B0001B4B0121029A99542800FFF71DFF0500C0
:1030C00080E70398FFF7B1FE411C0498FFF7D0FE9C
:1030D000059B1A4D049A2C601A60FFF7E1F8059BD6
:1030E0002C681B68002B02D0A6239B0201E09823CA
:1030F0005B026420B421E41A6043490203F0F2FE4B
:10310000B4225202030000920D49220007A806F0E3
:103110001DF907A800F0AAFF21B0F0BD6807002044
:1031200068060020680800200498020004300100AE
:103130005425002058250020642500206C0800201C
:10314000FCA70000F0B50020B7B00024FFF7D4FEC4
:10315000270005002600002D20D0FF226B6828687C
:103160009C460233FF1803120136134011009C42A3
:1031700000DA1C0002140A400392624601400192E8
:103180000091039A1C4904A806F0E0F804A800F096
:103190006DFF2800FFF7B0FE0500DCE7174D28683B
:1031A000FFF743FE3B00019000943200144904A84D
:1031B00006F0CCF804A800F059FF124B1C682B68ED
:1031C000002B02D0A6239B0201E098235B0264201F
:1031D000B421E41A6043490203F084FEB42252028F
:1031E000030000920849220004A806F0AFF804A8E2
:1031F00000F03CFF37B0F0BD32A8000068080020A6
:1032000046A800006C08002017A8000070B5002038
:10321000FFF70BFE04000120FFF707FE844200DAEF
:1032200004000A4B1E687542754128001D60FFF7B7
:10323000EDFD002E01D0064B00E0064B064A2800AB
:10324000611C1360FFF714FE70BDC04668080020C3
:1032500004300100049802006C080020F8B500203A
:10326000FFF7E3FD07000120FFF7DFFD3E00224DE1
:103270000643224C0CD180219820C9024002FFF75E
:10328000ABFD01213000FFF7F3FD2E601C4B2FE05A
:10329000874208DD0023A6212B60194B8902236099
:1032A0002368002011E0012380212B60154BC90207
:1032B0002360F5E71A68551C18D0120E522A07D160
:1032C00001205A68023292009B188B42F2D311E01F
:1032D000002800D023600C4C0C49200006F062F856
:1032E0002000FEF7A3FEFFF791FF04E0002802D0C4
:1032F000236000E02160F8BD680800206C08002011
:103300000430010004980200A02500207BA80000E2
:10331000F0B585B0039203220333DC1714402A4E24
:10332000E3189C10336801900291002B02D0802298
:10333000D20201E0A6229202244FA51C3B68AD00F8
:103340005B199A4217D2FFF719FE3368002B02D09F
:103350008022D20201E0A62292023B685B199A42C7
:1033600009D21B4C1B49200006F01CF82000FEF778
:103370005DFE002026E0029B3E681B06190C6B4692
:103380001A7BA423DB051343019A0B431104FF228C
:103390001204114019433000FFF756FD3300301D71
:1033A0000833210001933B60FFF74EFD002C04D051
:1033B0000A9A21000198FFF76BFD3000019B083D40
:1033C0005D193D6005B0F0BD680800206C08002064
:1033D000A0250020A4A8000010B5FFF7CFFD10BD68
:1033E00070B59AB0FFF73AFFFF22264CD2000021B9
:1033F000200005F0B2FB0020FEF7E0FE042804D117
:103400000020FEF7EFFE042831D00020FFF7A2FDD8
:10341000FF25002600281AD003681A142A400A2A19
:1034200008D11A122A40FF2A0ED0D200A1180B711F
:10343000A05009E0132A07D11B122B40FF2B03D009
:10344000DB00E2181671E650FFF756FDE2E7FF21B8
:103450000200C900235808305D1EAB41D2188842D3
:10346000F8D1094901A805F071FF01A802E0FFF7B2
:10347000CDFE064800F0FAFD054800F0F7FD1AB051
:1034800070BDC046CC1B0020CBA80000E7A8000000
:10349000DFA8000000220121094B5A60094A51604F
:1034A0005A68002AFCD00022C021054B49001A614D
:1034B000044B01329A60044B01325A501A60704733
:1034C000FC1000400010004000E100E00222064B2A
:1034D0000121DA670022054B5A61054A11615A69D8
:1034E000002AFCD07047C04604E100E0FC10004018
:1034F0000010004010B5054B1A781C00002A01D0BE
:10350000FFF7E4FF0023237010BDC046F808002039
:10351000024B18680123400018437047F40800204C
:10352000004870477C250020024B186801234000AA
:10353000184370473C01002070B504000D001600D0
:10354000FEF76CFD8023012200215B055B6E62703B
:10355000E270020AA271020CE2711A0A60716372CF
:10356000000EA2721A0C1B0E267025712072A1701B
:10357000E272237370BD0000124B10B51B68124C31
:103580005A1C0FD0114C002B0CD0114C012B09D020
:10359000104C022B06D00D4C042B03D00E4C052BE7
:1035A00000D10B4C21000D4805F0FCFE200005F079
:1035B00001FF0300042204339B0809481B01134345
:1035C000036010BD40010020B9A90000B2A90000AD
:1035D000C4A90000C9A90000BEA9000068250020F8
:1035E0006425002070B5214C2278002A3DD1204B63
:1035F00001215A608022D20511605A68002AFCD04D
:10360000002207201B4B1C4901255A5004395850F1
:1036100008315A5019481A4958501A491A485A50EC
:103620001A495A50A622D2009D50082218495A50D1
:10363000043158500220174958501748174958501C
:10364000174804395850182016495850C12189008C
:103650005A500539FF395A58083802435A50124A0D
:1036600012499950FFF716FF257070BDF808002029
:10367000FC000040001000400C05000074696275F9
:103680001C05000024050000200004022C05000099
:103690001405000034050000FFFF00003C05000099
:1036A00021100100540500000405000070080020EE
:1036B00010B500280EDD0C68E3070BD56410FF2C55
:1036C00008D8054B1B78002B01D1FFF78BFF034B6C
:1036D000034AD45010BDC046F8080020240500005D
:1036E0000010004013B5002815DD0C68E30712D563
:1036F000082209496846641005F026FA072C0AD802
:10370000064B1B78002B01D1FFF76CFF6B46044A78
:103710001957044BD15016BDAAA90000F808002083
:10372000001000400C05000010B5002813DD0C68E7
:10373000E30710D56410532C0DD8074B1B78002BD2
:1037400001D1FFF74FFFFFF7C1FEA123034ADB00C2
:10375000D450FFF79FFE10BDF80800200010004075
:1037600070B50E4B06001B78002B01D1FFF73AFF16
:1037700000200B4D2C7884420ED00A4B2022197861
:103780000323091B1940084B49015918300005F063
:10379000DBF90120013C2C7070BDC046F808002008
:1037A000F9080020F008002070080020002330B540
:1037B00089B0984226DD03240D682C409C4221D11B
:1037C0002300042D1ED90F212A681140062919D182
:1037D00012091F2A16D96846FFF7C2FF23000028E6
:1037E00010D06B46012019780123A14203DB6B4600
:1037F0001B5D5B000343A200AA1801345360202C18
:10380000F2D10423180009B030BD0000F0B5424BDE
:103810008BB01B78002B01D1FFF7E4FE02AD28002E
:10382000FFF79EFF002870D02B780B2B6DDD6B7897
:10383000012B6AD1EA780023012A66D1374F384C30
:103840003B6023712B79374A1360002B0ED115256D
:103850006D446A782878AB78120202431B04134344
:103860001A00EB781B0613433B6050E0012B10D18C
:1038700015266E4472783078B378120202431B0426
:1038800013431A00F3781A261B0613433B606A7C25
:1038900025E0022B02D16A7B162620E0042B0DD1F5
:1038A000152108226944684605F04EF900980199EF
:1038B00001F0CAFB04F0DEFF386028E0052B26D1BA
:1038C000152108226944684605F03EF900980199DF
:1038D00001F0BAFB04F0CEFF1E2638606A7D6E440C
:1038E000132A00DD13220023934204D0F05CE11878
:1038F00008710133F8E704200021E21804339B101B
:103900001B0103431171236003E0002001E000224A
:10391000E9E70BB0F0BDC046F8080020F40800202D
:103920007C2500204001002010B5041E26D0144B39
:103930001B78002B01D1FFF755FEFFF7C7FD0020D4
:103940001049114A114B8C50586001300860596879
:103950000029FCD000200D4908610A490130886027
:1039600019690029FCD00A4B0A491B785B01CB1866
:1039700004498B50FFF7AAFDFFF78CFD10BDC04630
:10398000F80800200010004004050000FC10004072
:10399000F00800207008002030B589B000281EDD36
:1039A00003230A6813401AD1042A18D90F2011687A
:1039B0000840062813D109091F2910D90124013311
:1039C000990051580020214201D04910C8B26D46DB
:1039D000591E6854202BF2D16846FFF7A5FF09B0A5
:1039E00030BD30B589B0002826DD0868830723D1B3
:1039F000042821D90F2302681340042B1CD1FEF7A1
:103A0000FDFC050005F0D6FC041E122C00DD12247E
:103A1000220002210D326846FFF78EFD6B465C7373
:103A20000023A34205DA1A00E95C6A44917301336A
:103A3000F7E76846FFF778FF09B030BD70B50C00B6
:103A400088B0012833DD0868830730D104282ED9D7
:103A50000F2302681340042B29D14B68DB0726D5BE
:103A6000FEF7CCFC060005F0A5FC646805006410B8
:103A70000E2800DD0E252A00012111326846FFF7CD
:103A80005BFD6B466A465C73231293732314D373F6
:103A90000023240E14745574AB4205DA1A00F15C4D
:103AA0006A4491740133F7E76846FFF73DFF08B0B9
:103AB00070BD30B589B0002814DD0C68E30711D55E
:103AC000102200216846FFF737FD6B466A466510F5
:103AD0005D73684663122D0E64149373D47315746A
:103AE000FFF722FF09B030BD184B10B55A681849CE
:103AF000002A03D000225A6001328A601B691448F0
:103B0000002B22D00023114A13618022D200845856
:103B1000104A012C16D1A923DB00C3585B42136065
:103B20000D4A1378032B01D80133137003220B487D
:103B30000378013313400A4A03705B01D318094A22
:103B40008B5000E0136001238B6010BDFC1000401F
:103B5000001000403C010020F9080020F00800207F
:103B6000700800200405000010B5034A0E21034828
:103B700000F0B4F810BDC046CC000020D0A9000071
:103B8000044A05491368C85401339B059B0D136013
:103B90007047C046000D0020FA080020114A70B599
:103BA0001368114C984211DA015D451CFA3901295C
:103BB00006D8AB4206DD2118497801391F2901D901
:103BC0002800EFE70100251A461C02D100231360EC
:103BD00006E0665C6E5401318B42FADC181A106004
:103BE00070BDC046040D00200C0D002010B5FEF77E
:103BF0000BFA064B1A68904201D200221A601B6829
:103C0000C01A034B83428041404210BD080D002082
:103C1000204E000010B5094C094A236812689342EF
:103C20000BD0084AD05CFEF733FB002805D0236890
:103C300001339B059B0D2360EDE710BD0C110020A7
:103C4000000D0020FA08002010B50400064B074ABA
:103C50001B6812689B1ADB439B059B0DA34202DA8B
:103C6000FFF7D8FFF2E710BD000D00200C11002077
:103C7000F7B506000191151E2FD05768B800441CF7
:103C80000630FFF7E1FFFB20FFF77AFF1C20FFF76C
:103C900077FFF0B2FFF774FFE0B22412FFF770FF76
:103CA000E0B2FFF76DFF6B461879FFF769FF00265A
:103CB000BE4212DAB300EB189C680136E0B2FFF79F
:103CC0005FFF2012C0B2FFF75BFF2014C0B2FFF706
:103CD00057FF200EFFF754FFEAE7F7BD70B5074D19
:103CE0002C68092C08DC0C236343054E01349851E1
:103CF000F31859609A602C6070BDC0461011002006
:103D000004260020F0B589B004900E0001284BDD98
:103D1000284B08680293830709D1042807D90F2389
:103D200002681340042B02D1FEF768FB0290214B7E
:103D300070680393830709D1042807D90F23026809
:103D40001340042B02D1FEF759FB039000271A4BB6
:103D50001A4D1B680593059B9F4225DA2B1F02997C
:103D6000186805F015FB00281BD12B686C680693BA
:103D70000190019B069A934213DA206803990794F5
:103D800005F006FB0834002807D131000498079B92
:103D900008315B680238984709E0019B01330193C1
:103DA000E7E701370C35D6E71B20FCF7CDFB09B060
:103DB000F0BDC04616A90000101100200826002002
:103DC00010B5FEF7FDFFFEF723FAFEF7B5FBFEF791
:103DD000EDFBFFF7C9FE00F019FD00F0D7FE10BDA6
:103DE000962210B512010021034804F0B6FE00220D
:103DF000024B1A6010BDC0466C120020CC0200209D
:103E0000064B074A1B6812689B1ADB439B059B0DF8
:103E10000122834200DC002210007047000D0020C8
:103E20000C110020F8B505000C0016001F1E0ED165
:103E30000320FFF7E5FF002827D0FA20FFF7A0FEB8
:103E4000E8B2FFF79DFEE0B2FFF79AFE1DE0501DBD
:103E5000FFF7D6FF002818D0FB20FFF791FEE8B24D
:103E6000FFF78EFEE0B2FFF78BFEF0B2FFF788FEA1
:103E70003012C0B2FFF784FE3C00E31B9E4204DD1B
:103E80002078FFF77DFE0134F7E7F8BD70B5002418
:103E9000F0250B4B1B689C420EDA2A006243094B4B
:103EA000D3181A78002A05D05978002311201A0057
:103EB000FFF7B8FF0134ECE7FFF792FF70BDC04693
:103EC000CC0200206C1200200123F3B50400FFB0E7
:103ED0000D0010001A420DD002AA1370431002A95F
:103EE000537042121B0E40148A700B71C8700B0085
:103EF000052273E0032313401ED1042A1CD90F228C
:103F000001680A40042A17D1023302AA1370FEF78F
:103F100075FA060005F04EFAF823FF33984200DDEB
:103F200018000023834205DA01335A1EB25C02A94D
:103F3000CA54F7E7421C50E0042801D0002809D1F8
:103F4000032302AA04381370434243415370130001
:103F5000022243E0002B45D1042843D90F210268F7
:103F60001140052912D1043302A90B70F82312095C
:103F7000FF3392009A4200DD1A00002393422BDAAD
:103F80000133C118C97802AEF154F7E7062929D1E7
:103F900001390E00120956430196F826019FFF369B
:103FA000B7421FDC02AE31700136934213DA0127AB
:103FB000013399004158394201D0394100E00A49A2
:103FC000012737700F127170B7700F14090EF77058
:103FD00031710536E9E7019A013202AB2900200070
:103FE000FFF720FF7FB0F3BD19FCFFFF70B5F02392
:103FF000050000240D4A1800604380184178A9424A
:1040000003D001340A2CF6D10FE0F022002104F095
:10401000A4FD074A1368013BA34200D114600023AA
:1040200029001A001120FFF7FDFE70BD6C12002060
:10403000CC02002010B5B2B002236A46040013700F
:1040400005F0B8F9C72800DDC7200023834205DA50
:10405000694601335A1EA25CCA54F7E7421C6B46FC
:10406000FE211420FFF7DEFE32B010BD30B5B3B034
:1040700002236A460500137005F09CF9041EC72C44
:1040800000DDC7240023A34205DA694601335A1E26
:10409000AA5CCA54F7E720003230FFF7D5FD621C56
:1040A0006B46FF211420FFF7BDFE33B030BD00008A
:1040B000F7B5234B06001B68F0200093002321492D
:1040C000009A93420ADA02005A438A185478B4429A
:1040D00002D11278002A31D10133F1E70024F02314
:1040E0001A00624301920199164A55182F78002F41
:1040F00006D001340A2CF3D11348FFF7B7FF1DE0B7
:10410000F0223900280004F028FD02230D4A01990D
:10411000EB6053540D4AF1008A58009B6E70AE70EC
:10412000AA602F616F61A34202DC054B01341C6061
:10413000002331001A001020FFF774FEF7BDC046BF
:10414000CC0200206C1200208BAA0000CC1B0020A7
:1041500010B5FFF79BFE0024064BE200D3181B7935
:10416000043B012B02D8E0B2FFF7A2FF0134FF2C81
:10417000F2D110BDCC1B0020F7B50E0000247F2526
:104180000190194BE200D1180979062901D00329C1
:1041900026D1985883682B401C2B21D1C3681A0064
:1041A0002A40042A1CD102692A40192A18D11B0A64
:1041B00001339B000C30C018FEF720F9070005F012
:1041C000F9F80023B0420BD19E4206DD019AF95C5A
:1041D000D25C914204D10133F6E7E0B2FFF768FF09
:1041E0000134FF2CCDD1F7BDCC1B002070B5FDF7FD
:1041F0000BFF184B1A68904201D200221A601A680D
:104200001549821A8A4223D918600020FDF7D6FF8B
:10421000444244416042072404430020FDF7E2FF8A
:10422000002810D0082600250C4BEA00D3181B7973
:104230009C4201D0B34202D1E8B2FFF739FF013509
:10424000FF2DF1D104E0631C02D001267642EAE79B
:1042500070BDC046FC0C00200F270000CC1B0020C6
:1042600037B500240500FFF711FE01A80194FDF702
:1042700093FF21002000FEF7C9FAFEF747FCFDF787
:10428000C5FFFDF7C4FFFEF795FDFDF7E9FEA5426A
:1042900004D0FEF713F80248FFF7E8FE37BDC0462A
:1042A000A0AA0000002310B501001A001120FFF79A
:1042B000B9FD10BD07B56B46197069465A701312E7
:1042C0008B701314120ECB700A716B46010005221D
:1042D0001320FFF7A7FD07BD10B50A00010012204B
:1042E000FFF7F2FD10BD70B5050008000C0032307C
:1042F000FFF7AAFC2B00220000211B20FFF792FDF4
:1043000070BD10B50C000300110014202200FFF74F
:1043100089FD10BD70B506000020FEF7EDFD0024FC
:10432000FF25002810D003681A142A40152A05D149
:104330001B122B40B34204D1040002E01D2A00D11D
:104340000024FEF7D9FDECE7200070BDF0B5802712
:104350009DB0FFF75FFCB64DB64C2868FF00391AD8
:104360002018FDF77BFF2B680600C3182B60002B7D
:1043700000D1D9E1002E0DDD2868391A2018FDF78B
:104380006DFF2B6806001B182B60FDF73DFEAA4B46
:104390001860EFE72378FA2B00D00CE12B68022B92
:1043A00006DCFFF723FC002800D1BDE10120B6E1C7
:1043B0006078A5780238182800D9FAE002F0FEFCEF
:1043C0000D1E22262932F93D67F96F83D4E5F9F9EC
:1043D000F9F9F9F9F9F9F9F9F300FF2D00D1E8E05D
:1043E0002800FFF703FE00229449EB005A50CB1837
:1043F0001A7129000092130013204DE02800FFF7E6
:1044000057FED6E02800FFF7F1FDD2E0FFF7A0FE4F
:10441000CFE0FFF73BFD0020FFF722FF8848FFF7C2
:1044200025FEC6E0632D00D9C3E0864BAA00D25812
:1044300029001520FFF748FDBBE000242000FFF70E
:1044400069FF071E03D10134642CF7D1B1E00830B5
:1044500004F0B0FF06000530FFF7F6FBFB20FFF786
:104460008FFB1D20FFF78CFBE0B2FFF789FBF0B25A
:10447000FFF786FB3012C0B2FFF782FB0025AE4289
:10448000E1DD7B19187AFFF77BFB0135F7E70021A7
:104490001D200B000A000091FEF73AFF89E0FDF7AE
:1044A000CDFD03AC684A64210090684B200004F005
:1044B0001BFF02232000237004F07CFF2300020076
:1044C0000021162073E000245C4AE300D558002D3B
:1044D00046D06B689E00701DFFF7B6FB2B000025D1
:1044E0003200083321000120FFF79CFC0020FEF77A
:1044F00003FD2E002F0000281DD0FF2103681A1293
:104500000A40A24214D11A140A400B2A07D10B40C8
:104510000DD0012B09D0022B00D103E108E0132AB2
:1045200006D100252E002F0002E0060000E0070063
:10453000FEF7E2FCDFE7002E04D03200012120006C
:10454000FFF796FB002D04D02A0002212000FFF780
:104550008FFB002F04D03A0000212000FFF788FBDA
:104560000134FF2CB0D124E00024FFF78FFC22009F
:10457000210000942300DA20FEF7CAFEFF2221006A
:10458000D2002E4804F0E9FA13E0012D02D1FEF723
:10459000D9FD0EE0022D02D1FEF71EFF09E0012039
:1045A000FFF75EFE05E0002329001A001A20FFF73E
:1045B00039FC0320B3E0FB2B00D0F7E62A68042A7D
:1045C00000DCEEE62679E078214B360206439E4277
:1045D00000DDEBE6331D9A4200DCE2E6E35CFE2BF5
:1045E00000D0E3E66378A578711E1B2B5DD004D85C
:1045F000012B08D0082B2DD090E01D2B64D058D370
:104600001E2B7BD08AE0FF2D00D187E02800FFF72A
:10461000EDFC67790634B31E290000943A000A20A5
:10462000FEF776FE054BED00E8505D192F7175E041
:10463000040D00200C0D0020080D0020CC1B0020D4
:10464000AFAA0000C4230020C6AA0000C1AA00002F
:10465000F6030000632D61D86079022813D0032887
:104660001BD001285AD1A71D7A78A479BB781202F1
:1046700022431B0413431A00FB78AD001B061343AF
:104680005B0003430EE0002948DDB11EA01DFDF7CD
:1046900099FE264BAD00E85040E0A379AD005A1ECC
:1046A00093419B00214AAB5038E0601DFFF764FD49
:1046B00034E06279FF2D31D0022A2FD80634B31EA0
:1046C000009429000B2016E00B1E632B00DD6323F2
:1046D000002203A8934204DDA118497981540132D4
:1046E000F7E7D9430022C917194041180A70009012
:1046F000290015200133FEF70BFE0FE0012D0DD12F
:1047000000290BDD6379002B03D0322B02DD32232D
:1047100000E02B0064225343054A1360701DFFF72D
:104720003DFA01E0050003E71DB0F0BDC423002001
:10473000040000200122094B1A60094A1368002B6B
:10474000FCD00322074B1B68D8171040C018012368
:1047500080100638400018437047C04600C0004033
:1047600000C1004008C500400120704710B5064C4C
:10477000200000F041FB0549200000F061FB012210
:10478000034B1A6010BDC0463C110020801A060081
:104790001411002010B501210D20FDF753FC01215B
:1047A0000E20FDF74FFC00210F20FDF74BFC044CC1
:1047B000200000F05DFA1021200000F075FA10BD15
:1047C0002811002010B504680D20E30703D56410FC
:1047D000FF2C03D91720FBF7B7FE06E0FFF7DAFF3F
:1047E000E1B2024800F082FA002010BD281100203A
:1047F00010B5FFF7CFFF0021034800F077FA01233F
:104800004000184310BDC0462811002010B5034ACF
:1048100007210348FFF762FA10BDC0464801002097
:10482000CDAA00000D4B70B51B6804000E001500EA
:10483000002B01D1FFF79AFFE1B2094C200000F0F4
:1048400087FBF1B2200000F098FAE9B2200000F0F6
:1048500094FA200000F0E6FB70BDC0461411002061
:104860003C11002010B501240368234205D04168A3
:10487000214202D08268224201D10D2004E058106A
:104880004910802803D91520FBF75EFE0BE0FF29B5
:1048900001D91620F8E75210FF2A01D91720F3E7B3
:1048A000FFF7C0FF002010BDF7B501242300A04290
:1048B00037DD0A68144234D01B4B55101B684C6816
:1048C000002B01D1FFF752FF0127184EE9B230004B
:1048D00000F03EFB3C4205D03C413000E1B200F02C
:1048E0004CFA1AE00325254017D1042C15D90F23C3
:1048F00022681340062B10D113090193019B9D429E
:104900000BDAAB00E3185968394204D04910C9B238
:10491000300000F032FA0135F0E7300000F082FBA1
:1049200000231800FEBDC046141100203C110020D9
:10493000144B70B51B6805000E00002B01D1FFF76A
:1049400015FF114CEDB22900200000F001FBF1B27F
:10495000200000F012FA0021200000F005FB0028E2
:1049600001D040420CE001222900200000F0EBFAC7
:10497000200000F0F8F90028FAD0200000F0F8F943
:1049800070BDC046141100203C11002010B5012458
:104990000368234202D04168214201D10D2004E086
:1049A00058104910802803D91520FBF7CDFD07E0EA
:1049B000FF2901D91620F8E7FFF7BAFF400020438E
:1049C00010BD0000002370B5344D0400EB560133D8
:1049D0002BD10D211D20FFF7ABFF5A2804D1012256
:1049E0002A212A703D380AE00F211920FFF7A0FF85
:1049F000332807D102235F2220212B701A38FFF7BA
:104A000011FF12E00D211E20FFF792FFC7280AD1E7
:104A1000032300222A21A9382B70FFF703FF1B2252
:104A20002A211E20EBE700232B700023EB56022BDC
:104A300006D0032B13D0012B26D121001D2010E01E
:104A4000012C04D129211920FFF772FF0DE0032C5E
:104A500015D12B211920FFF76BFF043C05E0210045
:104A60001E200124FFF764FF64427F2801DD013826
:104A7000FF3803007F330ADA7F20404207E0052C2D
:104A800002D12D211920ECE7012400206442642387
:104A90007F21584302F026FA604370BD4401002094
:104AA00010B50120FFF78EFF01234000184310BD11
:104AB00010B50320FFF786FF01234000184310BD07
:104AC00010B50520FFF77EFF01234000184310BDFD
:104AD000F8B501263400B04236DD0F683E4233D0CF
:104AE0004D68AB0730D1042D2ED90F232A6813400F
:104AF000062B29D1154B1B68002B01D1FFF736FE81
:104B00000024354204D12B681C09202C00D9202414
:104B10000F4E7F10F9B22200300000F014FAA70007
:104B2000EF19AF420DD0300000F01DF90028FAD087
:104B3000300000F01DF9012340001843686004357F
:104B4000EFE70120640004432000F8BD14110020A9
:104B50003C11002000207047002070470020704763
:104B600000207047002070470020704700207047E9
:104B700000207047002070470020704700207047D9
:104B800000207047704770477047000010B5034A17
:104B90000C210348FFF7A2F810BDC0468001002099
:104BA0000EAB000010B5FDF73FFB0648FDF7AAFB72
:104BB000FFF706F90448FFF759FAFEF711FCFFF773
:104BC000C7FA10BD4605000084AB000010B5FDF724
:104BD000B5F910BD70B5002504AC24780573A94261
:104BE00005D10A4B0A4A23210A4803F02DFF016030
:104BF0000949920052589B0002715B588371A300CF
:104C00005B58856043710223C37170BDD9AB00004E
:104C10009CAB0000E7AB000070AC0000037B002BF6
:104C200004D143738373036101330373704700003E
:104C30001FB50191A02100240068C900D2B24450E0
:104C4000012A07D0A24203D0032A05D1042202E0A0
:104C5000022200E006221343034A8350034B019AC9
:104C6000C250012343501FBD54050000240500001D
:104C700010B50400FFF7D2FFA1222368A179D2006A
:104C800099506179064A200099502179043299504F
:104C9000044B19685A689B68FFF7CAFF10BDC046ED
:104CA0000C0500001C1100204BB2002B0CDB8023F4
:104CB0003F290CD81F290CD80F290CD807290CD84C
:104CC00003290CD81B060BE080239B0408E0DB04BF
:104CD00006E01B0504E05B0502E09B0500E0DB0548
:104CE0000168014A8B507047240500000368074A99
:104CF00099501A00FC32D1680029FCD0A321C900C8
:104D000058580023C0B2D3607047C0461C0500004D
:104D100007B58022074BD2051A6000229A60023242
:104D20001A710F230C3200930349023B0348FFF72B
:104D300051FF07BD1C110020003000402811002049
:104D4000F8B505000E0017000024BC4208D02B68FF
:104D5000315D1B6828009847002801D00134F4E732
:104D60002000F8BD704710B51C3001F0CDFB10BD20
:104D700010B51C3001F0BAFB10BD70B5437E0D00BC
:104D8000002B05D06430040001F0CDFB002801D0D9
:104D9000002004E02000290001F099FB012070BDF3
:104DA00010B51C3001F0B6FB10BD0000F7B5019343
:104DB000FA23002504009B0083600D4B45600833F7
:104DC00003601C300F00160001F076FB20006430F9
:104DD00001F072FB074AB600B35827616375019B67
:104DE00020009B009B586576A576A375FEBDC04646
:104DF00050AC000070AC00000123A022C375837D7D
:104E00000C49C133FF33D2059B009950437DC13318
:104E1000FF339B009950CC210369074A49049950FC
:104E20000521243A9950817D08329950417D034AE9
:104E3000995070470C060000240500000C05000086
:104E4000A02302690020DB00D0500948814204D928
:104E50000848814204D9CD2103E0CC21490401E076
:104E60008021C904044811500521D1507047C04623
:104E7000A086010090D0030024050000F7B50500CE
:104E800000200C00019382425CD0161E402E00D9F7
:104E900040262F001C37380001F024FBB1222B697B
:104EA000D20080219C50012289005A50A97E0029FD
:104EB00001D11A621A600024731E2A69A34206D126
:104EC000019B002B03D0802302219B00D1500123A2
:104ED00013621300FC33D968002902D1996A0029B2
:104EE000F9D0996A00290AD1D960A323DB00D158EF
:104EF0003800C9B2013401F0EAFAA642DCD8019ABE
:104F00002B69002A04D11A00FC32916A00290AD0C8
:104F100001210022AA7659611900FC318868002815
:104F2000FCD08A6007E00121A976D961D16C002903
:104F3000FCD00021D164FC339A6A002A01D00022FF
:104F40009A62E0B2FEBD10B50123FFF797FF10BDD6
:104F50000300AC3310B504001970643001F0C2FADC
:104F60000123637610BD0000F8B500220D0001009A
:104F70004276AC31036904000878B121C900585069
:104F8000802189005A5001321A629A6026006436E4
:104F9000300001F0B9FA00280ED03000276901F086
:104FA000A5FA1E4BF8502369FC331A6A002A0CD16B
:104FB0009A6A002AF9D008E02369002D0AD11A0064
:104FC000FC32916A002905D10EE09A6A002AF3D1D9
:104FD0001A62DBE701225A611A00FC32916800294B
:104FE000FCD00021916006E00121D961D16C00293B
:104FF000FCD00021D1641A000020FC32916A814269
:105000000BD0074990625A5802305A50824204D05D
:10501000043A534253410230C01AF8BD1C05000047
:10502000C404000010B50121FFF79EFF10BD000071
:1050300010B51323142202490248FFF7B7FE10BD32
:10504000004000403C110020F0B5474680B4CB0F33
:1050500098464A4C4B005B0D1E1982B007000A00AF
:10506000132E35DC002E57DB454B040033411F0067
:105070000F4007430D00002F24D05B081C000C409C
:1050800020430027002807D0132E00D172E0802291
:10509000D202324199430A434346DE00394B1100A4
:1050A0009E1934687568380022002B0002F0DAF986
:1050B000009001910098019922002B0003F086F8DE
:1050C00004000D002000290002B004BC9046F0BD91
:1050D000332E0CDD802304000D00DB009E42F1D155
:1050E00002000B0002F0BEF904000D00EAE7264CB6
:1050F0000D00A446012463446442DC40A44661469A
:1051000004000142DED049080142C5D08027FF05D6
:105110001F4188430743BFE74B005B08034304007C
:105120000D00002BCED00B031B0B03435A4213433D
:1051300080221B0B120313404A0C52041343190024
:105140004346104ADB00D3181C685D6822002B0020
:1051500002F088F9009001910098019922002B003B
:1051600003F034F842464B005B08D6073343040093
:105170001D00A7E780273F0689E7C04601FCFFFF27
:10518000FFFF0F00F8AC0000EDFBFFFF30B5214A38
:105190004B0087B05B0893421EDD1F4A934205DD3A
:1051A00002000B0003F012F807B030BD02AA00F0B5
:1051B00035F803231840049A059B01281ED00228C5
:1051C00011D000281FD00298039900F02DFA8023F7
:1051D0001B069C466144E7E700230022009300235E
:1051E00000F088FFE0E7012402980399009400F0A2
:1051F00081FF80231B069C466144D5E702980399F2
:1052000000F012FAD0E7012402980399009400F00C
:1052100071FFC9E7FB21E93FFFFFEF7FF0B54E4685
:1052200057464546E0B4DC4B4E0090B01700894627
:1052300076089E4200DC81E0D84B9E4220DCD84AB2
:10524000002900DC89E1D74B02F0C0FFD54B0400F8
:105250000D009E4200D18AE0D34AD44B02F0B6FF43
:1052600002000B0020003A607B60290002F0AEFFD4
:10527000CD4ACE4B02F0AAFFB860F960012066E08B
:10528000CB4B9E4200DC8DE0CA4B9E4265DCCA4996
:1052900032158A46924453461B05F51A290004002C
:1052A00003F0E8FA03F01CFB02000B0020002900C9
:1052B0000A920B9302F08AFF0022C04B02F00CFD11
:1052C0000290039103F0D6FA03F00AFB04000D00EC
:1052D00002000B00029803990C940D9502F076FFE2
:1052E0000022B64B02F0F8FC002200230E900F9132
:1052F00001F002FF002800D14CE100230022200031
:10530000290001F0F9FE0222431E9841131AAC4A0B
:105310003900019202220AA80092524600F09EFA39
:105320004B46002B13DA8022120694467B684042DB
:1053300063447B60FB686344FB6008E002000B0091
:105340003A607B60002200230020BA60FB6010B04E
:105350001CBC90469946A246F0BD02000B0002F02C
:1053600035FFB860F960386079600020EFE7D3223C
:105370008E4B520502F02AFF924A934B04000D0017
:1053800002F024FF02000B0020003A607B6029003D
:1053900002F01CFF8B4A8C4B02F018FFB860F960DA
:1053A0000120D4E700F056FF884A894B04000D0025
:1053B00002F092FC0022874B02F054F803F05AFAF4
:1053C000804603F08DFA764A764B0690079102F0FC
:1053D00083FC02000B002000290002F0F7FE734B53
:1053E00002900391069807996F4A02F075FC4346B4
:1053F00004000D00049405951F2B30DC013B764A18
:105400009B009B589E422AD002000B0002980399F1
:1054100002F0DCFE02000B0005000C003A607B602D
:10542000029803992A00230002F0D0FE049A059BFB
:1054300002F0CCFE06000B003200BA60FB604B4667
:105440004046002B00DB82E780231B069C46644419
:1054500061443D607C60BE60F960404277E7049A39
:10546000059B0298039902F0B1FE0B0002003A601E
:105470007B604B0036155B0D05000C00F31A102BFA
:10548000CEDD06980799D322484B520502F024FC42
:1054900004000D0002000B000298039902F096FE32
:1054A00002000B00029803990892099302F08EFE05
:1054B00022002B0002F08AFE04000D0006980799D6
:1054C000404A414B02F008FC22002B0002F07EFE15
:1054D00002000B00049005910898099902F076FEED
:1054E00002000B003A607B604B005B0DF61A050072
:1054F000089A099B0C0002920393312E90DD0698C6
:105500000799B822304B920502F0E6FB04000D002B
:1055100002000B000298039902F058FE0A000100F5
:1055200013000291039202000898099902F04EFEBE
:1055300022002B0002F04AFE04000D000698079995
:10554000264A274B02F0C8FB22002B0002F03EFE49
:1055500002000B000492059358E7124B01F082FF02
:10556000104B04000D009E423CD00F4A0F4B01F03F
:1055700079FF02000B0020003A607B60290002F0F6
:1055800025FE094A094B01F06DFFB860F960012062
:105590004042DCE60323BAE6FB21E93F7BD9024027
:1055A00000004054FB21F93F3163621A61B4D03DE1
:1055B000FB213941FFFFEF7FEAFBFFFF0000704155
:1055C00088AD00007370032E8A19A33B83C8C96D90
:1055D000305FE43F0000E03F08AD0000C1492025F6
:1055E0009A837B39D3220D4B520501F03BFF0C4AC5
:1055F0000C4B04000D0001F035FF02000B002000F1
:105600003A607B60290002F0E1FD054A054B01F09C
:1056100029FFB860F9600120404298E661B4D03DAE
:105620007370032E8A19A33BF0B54F464646C0B4AB
:1056300087B000920193754B4F00814688467F08E2
:105640009F4263DC03F016F9002800D1DAE04A46F5
:1056500043464846414602F03FFB04000D006C4AB9
:105660006C4B02F039FB6C4A6C4B01F0FBFE2200E4
:105670002B0002F031FB6A4A6A4B02F0A7FD2200C0
:105680002B0002F029FB684A684B01F0EBFE220078
:105690002B0002F021FB664A664B02F097FD2200C8
:1056A0002B0002F019FB644A644B01F0DBFE220080
:1056B0002B0002F011FB029003910022604B2000AE
:1056C000290002F009FB029A039B06000F0020004C
:1056D000290002F001FB009A019B04000D004846DE
:1056E000414602F0F9FA02000B002000290002F006
:1056F0006DFD02000B003000390002F067FD020072
:105700000B0000204F4902F061FD70E002000B0029
:1057100002F0E2FA04000D003D4A3E4B02F0DCFAD2
:105720003D4A3E4B01F09EFE22002B0002F0D4FACF
:105730003B4A3C4B02F04AFD22002B0002F0CCFA1F
:10574000394A3A4B01F08EFE22002B0002F0C4FAD7
:10575000374A384B02F03AFD22002B0002F0BCFA27
:10576000354A364B01F07EFE2B00220002F0B4FADF
:10577000354B029003919F429FDD344B00229F42A4
:105780003ADC334900207B182E4916001F0002F036
:105790001DFD049005910022294B2000290002F0F4
:1057A0009BFA32003B0002F011FD029A039B0600B7
:1057B0000F002000290002F08FFA009A019B0400DC
:1057C0000D004846414602F087FA02000B00200017
:1057D000290002F0FBFC02000B003000390002F04F
:1057E000F5FC02000B000498059902F0EFFC07B0ED
:1057F0000CBC90469946F0BD164B002604920593CA
:10580000154FC8E700200F49F1E7C046FFFF3F3EB4
:10581000D43888BEE9FAA8BDC4B1B4BD9EEE213E1D
:10582000AD529C804F7E923E9015CB19A001FA3E5E
:105830007751C1166CC1563F4C5555555555A53F2E
:105840000000E03F0000F03F3233D33F0000E93F6B
:105850000000E0FF0000E73F0000D23FF0B55646F1
:105860004D4644465F46F0B48E4CA544099119005C
:105870001400A89A0B938C4B9200D2580B00029004
:10588000013BE01E18211D0016000892009301F054
:1058900029FBC3430200DB171A4013001100013338
:1058A0000E929A009B1ADB001B1906934C1B76196B
:1058B00018D4A99BA5009C46361926AF654401362D
:1058C00007E0286803F00CF8013403C70435B4423C
:1058D00008D0002CF5DA00200021013403C704357C
:1058E000B442F6D1089B002B01DA00F0F9FB76AB4D
:1058F00019008B4626AA9146089A0A930132D200D3
:105900009344029A9A469046009BDB0099440833E0
:105910009844009B002B00DAB5E14C460026002796
:10592000029D2268636803CD02F0D6F902000B00E5
:105930003000390001F096FD083C06000F00454597
:10594000EFD15346C0C39A4608239C46E144DA454A
:10595000DFD10899554A0B00944663449B0012A876
:1059600084461A000298624483460D920B9A0433CF
:10597000D200634493440F930591059A0A98D3008B
:1059800019000C938C46030063441E685F68002A6C
:1059900034DD12AB99461300454A80469446634471
:1059A000DB00984474AB9A460022424B3000390029
:1059B00002F092F902F05EFF02F092FF00223E4BED
:1059C00004000D0002F088F902000B0030003900DD
:1059D00002F0FCFB02F04EFF4B4601C399464346E2
:1059E00020001A685B68290001F03CFD08235B4237
:1059F0009C46E04406000F00D045D5D1069B300000
:105A00001A003900994600F0C1FCFF2300229B05D3
:105A100004000D0002F060F900F020FC0022274B8A
:105A200002F05AF902000B002000290002F0CEFB20
:105A300004000D0002F01EFF804602F051FF02003C
:105A40000B002000290002F0C1FB4C4606000F00AD
:105A5000002C00DCF8E0059B18205A1E920012ABC7
:105A60009B58001B19000141884481405B1A12A910
:105A70008B501722121B13410793079B002B4BDD02
:105A800001239C46059BE044002B00DCF2E28025CC
:105A90001096119712AB0021002409486D04059F50
:105AA00019E0C04684FDFFFF90AE0000FEFFFF3FFF
:105AB000FFFFFF1F0000703E00007041000020400B
:105AC000FFFFFF00002A02D0AA1A1A600134013138
:105AD00004338F4209DD1A68002CF3D0821A013199
:105AE0001A60012404338F42F5DC109E119F069B3F
:105AF000002B0EDD012B00D1B1E0022B09D1059B5B
:105B000012A95A1E920012AB9B5810939B029B0A3B
:105B10008B50079B022B7ED00023002230003900DF
:105B200001F0EAFA059B002800D16BE208995A1EA1
:105B3000914210DCBF490F988C4612A963448C46F1
:105B400000219B0063441C68043B21438342FAD13B
:105B5000002900D0B5E0089B12AA013B9B00D35856
:105B6000002B00D084E201220D9B043B59680132D6
:105B70000029FAD005990B008C4601336244079244
:105B8000934242DC0E9A9446A99A634492460B9A39
:105B90009B00944626AA90469A44059B0A9A634421
:105BA000DB0098440C9B94469946079BE144DB003C
:105BB000634405935346186802F092FE434618600A
:105BC0005960009B002B23DB444600260027029DE2
:105BD0002268636803CD02F07FF802000B003000FA
:105BE000390001F03FFC083C06000F005D45EFD195
:105BF0004B469E60DF6004239C460433E2449C468F
:105C0000059BE144E0449945D4D1079B0593B4E654
:105C100000260027ECE732003B000020864902F016
:105C2000D5FA06000F00002C00D175E7069A002077
:105C3000814900F0ABFB02000B003000390002F09C
:105C4000C5FA06000F0067E7069B002B12D1059BE3
:105C500012AA013B9B00D558EB1507930DE7059B56
:105C600012A95A1E920012AB9B5810935B025B0A5A
:105C70008B504EE70022714B01F062FA00280ED1E2
:105C80000023079348E7534600260027C0C39A46DF
:105C900008239C46E144DA4500D03AE659E6012360
:105CA0009C4601330793059BE044002B00DDEEE6A4
:105CB00032003B000020604902F088FA06000F0025
:105CC0002AE743460B93069B12A8183B190006933C
:105CD0009300C3580092002B0FD1564813008446FE
:105CE00012A8634484469B006344043B5868013A0D
:105CF00018390028F9D000920691069A00204E49E2
:105D000000F044FB009B04000D00002B00DAB3E11F
:105D100012AA94469F00DB0067449C460A9A0593AA
:105D2000624493461600386802F0DAFD22002B0028
:105D300001F0D2FF424B3060716000222000290048
:105D400001F0CAFF083E74AB04000D00043FB342EB
:105D5000E9D100239A464EAB0293089B99464B46E5
:105D600000260027002B21DB8020364B5D4698461D
:105D7000C005354900260027002408E008239C467A
:105D80000835E044A24511DB4346186859682A6883
:105D90006B6801F0A1FF02000B003000390001F038
:105DA00061FB013406000F00A145E7DA029A534671
:105DB0009446DB0063441E605F6001239C46093B00
:105DC000E2449C4674ABE3449B45C8D1029B994690
:105DD000A89B022B00DD82E0002B37DC1DD1059B48
:105DE00000254B441E0000243268736828002100FF
:105DF00001F038FB009B05000C00083E5A1E009283
:105E0000F2D2079B002B03D080231B069C466444E0
:105E10002A00230009990A604B6007200B9B184059
:105E20009F239B009D443CBC90469946A246AB46AE
:105E3000F0BDC046FFFFFF3F0000F03F0000E03F25
:105E40000000703EA0AE0000FB21F93F059B002042
:105E50004B441E0000214CAF32687368083E01F0CD
:105E600001FBBE42F8D1079B002B24D08023099A66
:105E70001B06CB18106053600B0002004E984F9920
:105E800002F0A4F9009B002B0BDD012450AD0CCDDA
:105E900001F0E8FA009B0134A342F8DA079B002BDB
:105EA00003D080231B069C4661440B000200099925
:105EB0008A60CB60B1E702000B00099C226063603E
:105EC0000B0002004E984F9902F080F9009B002BC6
:105ED000DBDC0B00020009998A60CB609DE7A89B80
:105EE000032B9AD1009B002B00DCE3E07E4A059B4C
:105EF00094464B441E685F68009B63449A46DB00EF
:105F00004B4498464CAB9B4643465C681B68180064
:105F1000210032003B000290039101F0A3FA04003B
:105F20000D0002000B000298039902F04FF93B00AC
:105F3000320001F097FA43469860D9601C605D60BA
:105F400008235B429C46E04426002F00C345DBD17A
:105F5000009B012B00DCADE0059BC8464B441E684E
:105F60005F685346DB009B46D844434630005C687C
:105F70001B683900009301941A00230001F072FAA3
:105F800004000D0002000B000098019902F01EF9B8
:105F90003B00320001F066FA43469860D9601C600D
:105FA0005D6008235B429C46E04426002F00C1450B
:105FB000DBD15D460027002408354D4450AE2A68E9
:105FC0006B683800210001F04DFA083D07000C0015
:105FD000AE42F4D1079B002B71D0099A4E994B46E3
:105FE0001160802109068C465B6849466344536012
:105FF0004B46DB688968634464449160D3601761F1
:1060000054610AE7994643460B93069B30005A4277
:10601000390000F0BBF90022344B04000D0001F000
:106020008FF8002832D0324B00222000290001F0E6
:1060300053FE02F01FFC4A460600970002F050FC97
:1060400000222A4B01F048FE02000B00200029002C
:1060500002F0BCF802F00EFC12AAD0514A46069B90
:106060000132183300920693930012AAD65044E6E8
:1060700001227FE500243AE5A89B022B14DC002BCB
:106080000FDC00D0C9E600250024BAE64B4620000C
:1060900029009E0002F0EEFB12AB98514B46009394
:1060A0002BE600200021DEE64EAB9946A89B032B91
:1060B00000D0B2E6079B00270024002B8DD14E9A1A
:1060C0004F9B09990A604B604B469A68DB680092C7
:1060D00001938A60CB603A0023000A614B619CE621
:1060E00076AB0A9335E4C046FFFFFF1F0000704106
:1060F0000000703EF0B54F464646C0B487B00092EF
:106100000193464A4B00814688465B08934205DC72
:1061100002F0B0FB4146031E484666D04A4643465D
:106120004846414601F0D8FD04000D0002000B0076
:106130004846414601F0D0FD394A3A4B06000F006F
:106140002000290001F0C8FD374A384B02F03EF824
:1061500022002B0001F0C0FD354A364B01F082F9D8
:1061600022002B0001F0B8FD334A344B02F02EF828
:1061700022002B0001F0B0FD314B324A01F072F9E0
:106180000E9B02900391002B34D0009801990022BD
:106190002D4B01F0A1FD029A039B04900591300064
:1061A000390001F099FD02000B000498059902F0F6
:1061B0000DF822002B0001F08FFD009A019B02F0E8
:1061C00005F8224A04000D00214B3000390001F08F
:1061D00083FD02000B002000290001F043F90200BA
:1061E0000B004846414601F0F1FF07B00CBC904659
:1061F0009946F0BD02000B002000290001F06CFD63
:10620000124A134B01F0E2FF32003B0001F064FD43
:106210004A46434601F026F9E7E7C046FFFF3F3E06
:106220007CD5CF5A3AD9E53DEB9C2B8AE6E55A3E20
:106230007DFEB157E31DC73ED561C119A0012A3FBC
:106240001111813FA6F810110000E03F4955555546
:106250005555C53F49004B0819007047454AF8B5E8
:10626000564692464B005B0D9A444D465F46444667
:106270005246F0B4894605000C000E000700132AB0
:1062800022DC002A47DB52463B4B134198460B0069
:1062900042461340034311D0384A394B01F0E2F82B
:1062A0000022002300F042FF002805D0002C41DB33
:1062B0004E46434600279E43380031003CBC904682
:1062C0009946A246AB46F8BD5246332A08DD8023E4
:1062D000DB009A45F2D102000B0001F0C3F8EDE7B4
:1062E000284A9446012263445242DA4093460242CD
:1062F000E4D0224A224B01F0B5F80022002300F03E
:1063000015FF0028D8D0002C1ADB5B464E469F4371
:1063100038003100D2E7194A194B01F0A3F80022E6
:10632000002300F003FF0028C6D0002C16DB002756
:106330000026C1E7802352465B0313419944B7E727
:106340005346142B12D03423524601279B1A9F40E8
:106350007F19AF429B415B429944D6E764006408D1
:1063600025430027002DA7D0074EA5E7133B9C46E9
:10637000E144CAE701FCFFFFFFFF0F009C750088A6
:106380003CE4377EEDFBFFFF0000F0BF4B0070B533
:106390005B0D14000A00002B1AD14B005B0803436D
:1063A00015D00022224B01F097FC224B0A009C42A0
:1063B00022DB4B005B0D363B1F4DE318AB4220DC6C
:1063C000002B0DDD1D4C1B0522401A43110070BD32
:1063D0001B4DAB42F0D102000B0001F043F8F6E791
:1063E0001D00353518DA174B02009C420ADC0B0001
:1063F0001548164900F032F8134A144B01F06CFCB2
:10640000E5E702000B001248124900F027F8104A95
:10641000104B01F061FCDAE7084C363322401B05D3
:106420001343190000220C4B01F056FCCFE7C04685
:1064300000005043B03CFFFFFE070000FFFF0F804D
:10644000FF07000050C3000059F3F8C21F6EA501FA
:106450009C7500883CE4377E0000903C30B54A00D3
:10646000DB0FDB0752081A43110030BDF7B50600F9
:106470000D000C008B180193019B671B9C4207D0F9
:10648000336821781B683000984701340028F3D125
:106490003800FEBD70B505000C00081E07D002F0E4
:1064A00089FF2B6802005B6821002800984770BDB7
:1064B00010B5FFF7EFFF10BD10B54022002104001A
:1064C00002F04BFB002320002364636410BD3F23D4
:1064D000026C10B5541C2340446C9C4201D0815482
:1064E000036410BD0023036443647047436C026C73
:1064F000934206D03F21C25C01330B40436410003D
:1065000001E0012040427047036C406C181A00D52E
:1065100040307047436C026C934201D0C05C01E094
:10652000012040427047036C406C5A1C3F231340CB
:10653000181A42424241D0B27047000003210A4873
:1065400002680A430260094802680A430260084977
:10655000084A094B9B1A03DD043BC858D050FBDCAA
:1065600000F012F8F9F706FE24050040540500403B
:1065700074B1000000000020AC020020FEE7FEE73E
:10658000FEE7FEE7FEE7FEE72D4B10B51A78012A7D
:1065900019D12C4A1268120715D12B4AE024116830
:1065A000F0220800104021420BD12849096811420D
:1065B00009D12749274A11608021274A0902116021
:1065C00001E03028F1D01A78012A0DD11D4909685F
:1065D000090709D1F0201C4909680140402903D16D
:1065E0001A490968014223D01B68DBB2012B25D16F
:1065F000144B1B681B0721D1134B1A68F0231A4058
:10660000A02A04D1114A12681A4203D016E0D02AF7
:1066100014D1F7E7114B1A68012A03D1C022104B9D
:106620001A600BE00F4A1A601A68012AFCD1F5E7DC
:10663000C1218020C900C0054250D5E710BDC04629
:10664000E00F00F0E40F00F0E80F00F0EC0F00F0B6
:10665000DFFF07C004050040186C004000EC064056
:1066600014EC0640759300000120704710B50368D4
:106670001322DB69984710BD704700000369054A83
:106680009950FC331A6A002AFCD0002201201A62B9
:106690007047C0461C050000030010B55C331A7833
:1066A0001F2313400122110099400D4B0424D96788
:1066B000C221036989005C505A60DA60A02200217F
:1066C000D20099500122074952425A5006491430CB
:1066D0005A500C395A5008315A50FFF703FF10BD79
:1066E00004E100E00C0500001405000010B51430B2
:1066F000FFF70AFF10BD10B51430FFF70BFF10BDF8
:1067000010B51430FFF7F2FE10BD0000030070B5A5
:106710005E331C780269604BD45003005D331C78F3
:106720005E4BD450030061331C785D4B012C0CD1BF
:1067300005005F352E78A225ED0056510500603525
:106740002E78A125ED00565100E00024D450962368
:10675000DB00994238D996231B01994237D99623F9
:106760005B01994236D996239B01994234D9E123A2
:106770009B01994232D99623DB01994231D9E12319
:10678000DB0199422FD996231B0299422DD9E1238F
:106790001B0299422BD996235B02994229D9E12306
:1067A0005B02994227D9E1239B02994225D93D4BAF
:1067B000994224D9E123DB02994223D9E1231B0327
:1067C000994221D8384B21E09E23DB021EE09D2315
:1067D0001B031BE0354B19E0354B17E0EC239B0303
:1067E00014E0344B12E0344B10E0344B0EE0344BE9
:1067F0000CE0344B0AE0344B08E0344B06E08023D5
:10680000DB0403E0324B01E080235B0531490024C7
:1068100053500423243953501100FC31CC600C62D6
:10682000C1210134890014605C30946053500378B6
:106830001F202200D9B20840824080342648FF340D
:106840005BB20251002B13DA0F230B40083B234CA1
:106850009B089B001B1903242140A140FC348C4061
:10686000DD69A543C0248C4021002943D96111E092
:10687000194C9B089B001B1903242140A140C025F3
:10688000FC348C40AD005E59A643C0248C402100EE
:1068900031435951026070BD0C0500001405000021
:1068A0006C05000090D0030000D0BE0E00B01300B5
:1068B0000050270000A04E0000F0750000509D0021
:1068C00000F0EB0000903A0100E0D70100B0AF0308
:1068D00000705F072405000000E100E000ED00E02B
:1068E000F7B5009308AB1B7800250193FA23040049
:1068F0009B0083600E4B45600833036014300F002B
:106900001600FFF7D9FD23005C3327611E70009B42
:10691000084A9B00995823005D331970019B2000A1
:106920009B009A5823005E33DD701A70FEBDC0468E
:10693000E0AE000070AC0000036910B51A00FC3234
:10694000D2680400002A0AD0A322D2009958143039
:10695000C9B2FFF7BCFD00222369FC33DA6010BD29
:1069600010B50248FFF7E8FF10BDC046F411002043
:10697000162307B5022200930249013B0248FFF7A4
:10698000AFFF07BD00200040F41100207047000059
:1069900010B500F011F8FFF7F9FF012000F0F0F951
:1069A000FEF700F9FEF712F9024B002BFAD000E0D7
:1069B00000BFF7E700000000C421114A89005058C9
:1069C000104B0340C02000020343535080239139F1
:1069D0009B02FF39535013608023A3220021DB0563
:1069E000D20099500122A1209A60074BC000195093
:1069F000C120023180001950403019501A60704790
:106A000000E100E0FF00FFFF00100140014B1860B3
:106A10007047C046E8010020F7B50023202877D84A
:106A20003C4B8000C258042A14D006D8022A0DD04C
:106A30000ED80423012A14D069E0062A0ED00BD305
:106A40001A2A0DD002231B2A0BD060E0082308E08D
:106A5000102306E0202304E0402302E0802300E02E
:106A600001232D4A1268082A04D9092A05D00A21CF
:106A7000022404E00821002401E011000124A025E3
:106A800001261C272548ED004651254D254E2D6831
:106A90001B02AD003D400195234D2D6800958559A1
:106AA000AC466746214D3D401D4385518359C02565
:106AB0009C46009BAD021D40FF2367461B023B40E6
:106AC0002B43019D1D43009B5F0160231F402B0052
:106AD0003B431C4301238451154C036063680F48FA
:106AE000002BFBD00024124B01255C60A123DB00AE
:106AF000C3584560A025ED0044511BB2914207D018
:106B000002D98A1AD34003E0521A934000E00023CE
:106B10001800FEBD70AC0000EC01002000700040C9
:106B2000E401002004050000E0010020FF00FFFF59
:106B3000FC700040F0B520286CD8374B8000C2585C
:106B4000364B1E68002E2ED1C2243548A4000759AA
:106B5000344B03253B40C0273F023B430351802376
:106B6000893C9B00FF3C03512F4F03602F4B803C1F
:106B7000D859FF3CA043D8510437D859A8432043E3
:106B8000D8510837D8590C35A843083D2843D85167
:106B9000A820C0001E508026C120760280001E5012
:106BA0001C601E4B1C6000231426214834005C43EB
:106BB000255804006F1C0FD1142058432250A020E8
:106BC0000325C132FF329200C0051550194A080052
:106BD0001268082A03D10BE0AA4218D1ECE7082A70
:106BE00002D9083AD14002E00820821A91400800F8
:106BF00014225343E3189A680C495132FF32920031
:106C000058605050DA68C1239B00CA5002E001333B
:106C1000032BCBD1F0BDC04670AC00005812002051
:106C200000E100E0FF00FFFF0405000000900040CD
:106C3000F0010020E80100201E4BF0B5596C18004F
:106C40001D4A002914D0A025A12600230124ED050A
:106C5000F600D1584F1C06D0D7187F68002F02D0FD
:106C600027008F40AF5114333C2BF2D100234364F3
:106C7000131DA02540329446002001240F4EED053F
:106C8000DA680F49920057180A495218526C002AC4
:106C90000CD01A1F1268511C05D01968FF2902D0A8
:106CA00021009140A9513A00FC32506414339C45B4
:106CB000E6D1F0BDFC900040F00100200C05000082
:106CC0000090004000B5202816D80C4A83009B583D
:106CD000032911D8A0220800C133FF33D2059B003D
:106CE00000F06CF802080406002104E00C2102E028
:106CF000042100E00321D15000BDC04670AC00006B
:106D000020280DD8074B8000C058A0220123D205AF
:106D10008340002901D1044901E0A121C900535059
:106D20007047C04670AC00000C0500000300002056
:106D3000202B0AD8A222A021D200C9058858034AD4
:106D40009B009B58D84001231840704770AC00004E
:106D5000084A0949094B10B51B688858FA22190AD4
:106D60001B0618439200002300F0F4F94904C00BFD
:106D7000084310BD04050000001001405C12002013
:106D800070B5041E09D0FFF7E3FF050000F014F80A
:106D9000FFF7DEFF401B8442F8D870BD0022044B91
:106DA0009A60044A13680133DBB213607047C0462F
:106DB000FC1001405C1200207047000002B47146D4
:106DC00049084900095C49008E4402BC7047C0462E
:106DD000002243088B4274D303098B425FD3030A1A
:106DE0008B4244D3030B8B4228D3030C8B420DD32D
:106DF000FF22090212BA030C8B4202D312120902BB
:106E000065D0030B8B4219D300E0090AC30B8B42F8
:106E100001D3CB03C01A5241830B8B4201D38B03A6
:106E2000C01A5241430B8B4201D34B03C01A52414B
:106E3000030B8B4201D30B03C01A5241C30A8B428E
:106E400001D3CB02C01A5241830A8B4201D38B0279
:106E5000C01A5241430A8B4201D34B02C01A52411D
:106E6000030A8B4201D30B02C01A5241CDD2C3098F
:106E70008B4201D3CB01C01A524183098B4201D30B
:106E80008B01C01A524143098B4201D34B01C01AF6
:106E9000524103098B4201D30B01C01A5241C3086E
:106EA0008B4201D3CB00C01A524183088B4201D3DD
:106EB0008B00C01A524143088B4201D34B00C01AC9
:106EC0005241411A00D20146524110467047FFE735
:106ED00001B5002000F0F0F802BDC0460029F7D04F
:106EE00076E7704703460B437FD4002243088B426A
:106EF00074D303098B425FD3030A8B4244D3030B41
:106F00008B4228D3030C8B420DD3FF22090212BA05
:106F1000030C8B4202D31212090265D0030B8B4281
:106F200019D300E0090AC30B8B4201D3CB03C01A6B
:106F30005241830B8B4201D38B03C01A5241430B46
:106F40008B4201D34B03C01A5241030B8B4201D336
:106F50000B03C01A5241C30A8B4201D3CB02C01AA1
:106F60005241830A8B4201D38B02C01A5241430A19
:106F70008B4201D34B02C01A5241030A8B4201D308
:106F80000B02C01A5241CDD2C3098B4201D3CB01AF
:106F9000C01A524183098B4201D38B01C01A52415E
:106FA00043098B4201D34B01C01A524103098B4262
:106FB00001D30B01C01A5241C3088B4201D3CB004D
:106FC000C01A524183088B4201D38B00C01A524130
:106FD00043088B4201D34B00C01A5241411A00D2E0
:106FE00001465241104670475DE0CA0F00D0494249
:106FF000031000D34042534000229C4603098B42B9
:107000002DD3030A8B4212D3FC22890112BA030A40
:107010008B420CD3890192118B4208D389019211C2
:107020008B4204D389013AD0921100E08909C30947
:107030008B4201D3CB01C01A524183098B4201D349
:107040008B01C01A524143098B4201D34B01C01A34
:10705000524103098B4201D30B01C01A5241C308AC
:107060008B4201D3CB00C01A524183088B4201D31B
:107070008B00C01A5241D9D243088B4201D34B0036
:10708000C01A5241411A00D20146634652415B1078
:10709000104601D34042002B00D549427047634659
:1070A0005B1000D3404201B5002000F005F802BD9E
:1070B0000029F8D016E770477047C046D0400B1C37
:1070C0001141203A03D49C4613411843634652426F
:1070D000934018437047C0468446101C62468C4655
:1070E000191C634600E0C0461FB500F08BFD002868
:1070F00001D40021C8421FBD10B500F0DFFC4042A2
:10710000013010BD10B500F07DFD002801DB00202E
:1071100010BD012010BDC04610B500F073FD002861
:1071200001DD002010BD012010BDC04610B500F0EB
:1071300005FD002801DC002010BD012010BDC04667
:1071400010B500F0FBFC002801DA002010BD012082
:1071500010BDC046F0B54F464646C0B41604360CC6
:107160009946330005042C0C070C150C63437E4331
:107170006F4365431C0CAD1964199C46A64203D9A4
:1071800080235B02984647446346250CEF191D0493
:107190004B464A4343432D0C240464199918C919DA
:1071A00020000CBC90469946F0BDC046F0B557464D
:1071B0004E4645464300E0B446028846760A1F0E16
:1071C000C40F002F47D0FF2F25D0002380259A46DB
:1071D0009946F600ED042E437F3F434642465D024A
:1071E000D20F5B006D0A1B0E904640D0FF2B39D0AA
:1071F00080220020ED00D20415437F3BFB1842465D
:107200005746591C62408C4607430F2F5CD86F4984
:10721000BF00C9598F46002E45D108239A46063B28
:107220009946DAE7424602282DD0032800D1C3E070
:10723000012800D0A2E0002500260240D4B2760248
:10724000ED05760A2E43E407264330001CBC904629
:107250009946A246F0BD002E1AD104239A46033B5C
:107260009946BAE72A00511E8A41901CC6E70120C0
:10727000002DC3D0280001F0C9FB431F76309D408C
:1072800043420020BAE70124FF2514400026D6E738
:10729000300001F0BBFB431F9E4000237630474285
:1072A0009A46994699E70C239A46093B994694E7F2
:1072B00080260024F603FF25C1E735004846B2E7E3
:1072C000350022004846AEE72904090C0800370CB7
:1072D0003604360C2C0C7943704367437443060C18
:1072E00064183619B14203D98021490288464744BF
:1072F0000004000C310409188D01681E8541890EB7
:107300002943350CED19AD010D43290104D50123A5
:1073100069081D4063460D4319007F31002925DDB2
:10732000680704D00F202840042800D00435280125
:1073300003D5274980330D401900FE29A3DC012421
:10734000AD016E0A1440CDB279E78020C003064239
:1073500007D0054205D128434602760A4446FF2558
:107360006DE706437602760AFF2568E70124611A75
:107370001B2905DD14400025002660E76346CBE7A6
:107380002E002023CE40591A8D406B1E9D412E4366
:10739000730704D00F233340042B00D0043673014D
:1073A00004D5012401251440002648E70124B60134
:1073B000760A1440002542E780260124F6032E4376
:1073C0007602760A1440FF2539E7C04610AF000068
:1073D000FFFFFFF770B5002830D0C317C5185D4018
:1073E000C40F280001F012FB9E231B1A962B0DDC04
:1073F0009622D21A95406A02520AD8B25202C005A9
:10740000520AE40702432243100070BD992B19DC95
:107410009922D21A9540124A2A40690704D00F21B6
:107420000D40042D00D00432510103D50C4B1A40FD
:107430009F231B1A9201520AD8B2DFE700240020D2
:107440000022DBE705222E00121AB921D6402A00BD
:10745000C91A8A40551EAA4135001543DBE7C046CC
:10746000FFFFFFFBF8B556465F464D464446F0B475
:107470000F00FD0FAA4609037C002E005F00450F98
:10748000490A7F0D2943C5001803BC46400A570F1F
:10749000640DDB0F3843D2009A4500D1AAE066465E
:1074A000A61B002E00DCFFE06346002B39D1030051
:1074B000134300D0D9E06B0709D00F232B40042BD6
:1074C00005D02B1DAB42AD416D4249191D000B0289
:1074D00000D482E0CA4B01349C4200D1FEE00A0095
:1074E0005646C84BED081A40500764055202054342
:1074F000120B640D002112030B0D1B056405120B0A
:107500001A436308C04CF60714401C436400640827
:107510003443280021003CBC90469946A246AB4625
:10752000F8BDB74B9C42C6D080231B041843382EAD
:1075300000DDEBE01F2E00DD1EE120239B1B9C469F
:1075400003006746BB40984613004746F3403B4361
:107550006746BA40571EBA4113430200F240EB1A85
:107560009D42B6411D008A1A7642911B0B0231D50D
:107570004A02560A002E00D1B4E0300001F046FA6B
:107580000300083B1F2B00DDB5E020222900D21AA2
:10759000D1409E400A009D4032439C4200DDB1E054
:1075A0001C1B631C1F2B00DDD5E0202114002800CC
:1075B000C91A8C40D8408D400443DA40681E85418A
:1075C00011002543002476E74146314300D134E2DF
:1075D000310045466B0700D06FE756464807ED0877
:1075E000C9080543864B9C4235D00A036405120B3B
:1075F000640D7FE76346E31A9B46002B00DC8BE0BB
:107600006746002F3CD07E4FBC4200D153E7802715
:107610003F0438435B46382B00DCF7E00243501E42
:1076200082410020D2B253194218AB4289411D0059
:10763000494289180B02CDD5714B01349C4200D1CF
:107640003DE101206F4A6B080A4028401843D507E6
:10765000054351082FE72B000B4300D1CBE18023DA
:107660001B030B431A03120B44E7013E002E6DD19E
:10767000AE1AB5429B41091A5B42C91A350075E73B
:107680000700174300D116E701235B429C46E34401
:107690005B46002B00D0E0E0AA18AA429B410918E3
:1076A0005B4259181500C5E7002E75D1661C76059A
:1076B000760D012E00DCF3E0AE1AB0464545BF4121
:1076C0000E1A7F42F61B370200D48FE0551BAA42E8
:1076D000B641411A76428E1B9A464BE75646002227
:1076E000002507E7280001F091F920300300083B4E
:1076F0001F2B00DC49E72A002838824000259C42E5
:1077000000DC4DE73F49E41A1140D4E60243501E25
:107710008241D3B2002222E7002B00D0F3E0631CA9
:107720009C465B055B0D012B00DC9FE0344B9C45C8
:1077300000D1C3E0AA180918AA428041404241186A
:10774000CD075208154349086446B4E62C4B9C42C9
:1077500000D0ECE6AFE611001F3CE1400C00202B0E
:1077600000D17FE04021CB1A9A4015436A1E954113
:107770000021254300242DE733000700203BDF4094
:107780003B00202E70D04027BE1BB0400243501E4D
:10779000824113430022E2E6002C4FD0184CA4454E
:1077A00000D1ABE08024240476422143382E00DD52
:1077B000DFE01F2E00DD43E12027BC1BA1460C00AB
:1077C0004F46BC40A0462C004746F4403C434F4641
:1077D000BD406F1EBD41F1402C43151BAA42924192
:1077E000411A5242891A64469A46BFE641464546C6
:1077F000314300D0BEE6002600240025F2E6C04654
:10780000FF070000FFFF7FFFFFFF0F801F2B59DCEA
:107810002027FF1ABC46070063469F405B46B946D7
:107820001700DF40B8464F4643461F4363469A4021
:10783000531E9A415B463A43D840F4E60C002C4371
:107840005CD0F643002E55D1551BAA42A441411AE3
:107850006442091B9A46644688E6964FBC4200D0B3
:10786000D8E628E6002280E700208FE70B002B43B4
:10787000002C00D0C2E0002B00D101E10300134333
:1078800000D118E6AB18AB42B64109187642711820
:107890000A0200D409E1884A1D00114064460AE644
:1078A000002C5BD10E002E4300D08AE00100114372
:1078B00000D1C2E0010015009A46FCE564460021B3
:1078C00000258FE620235B429C46DC44634607008C
:1078D000DF405B46BC46202B00D1ACE040235F4636
:1078E000DB1B98400243501E8241634613431A003B
:1078F000002098E66F4CA44500D057E70100150022
:1079000064469A46D7E5002C39D10C002C436ED042
:10791000DB43002B1AD0674CA44568D0382B00DD20
:10792000A4E01F2B00DDAEE020240F00E41AA740E6
:10793000B9462F00DF40B846A3464F46444627438A
:107940005C46A5406C1EA541D9403D43AD1895420B
:107950009B4109185B42591864466BE60C002C43A6
:1079600015D1010011437BD0010015009A46514CFE
:10797000A1E50D43691E8D410021ECB22DE74D4C70
:10798000A44534D0802424045B422143C6E704008C
:1079900014434ED0ED084C072C438025C9082D0315
:1079A000294208D0C6082E4205D1D208410711430A
:1079B0000C009A463100620FC900E50011433D4CAE
:1079C00079E50600164300D175E5AE1AB046454587
:1079D000BF410E1A7F42F61B370200D4F4E5551B57
:1079E000AA42B641411A7642891B9A4663E50100D4
:1079F000150064465FE5002200257BE5002B3BD0A7
:107A00000300134315D0ED084B072B438025C9080D
:107A10002D03294207D0C4082C4204D141070B0092
:107A20002100D2081343C9005A0F1143DD00214C35
:107A300041E5204C3FE5002054E700260025D1E534
:107A400034000F00203CE7403C00202E2BD0402784
:107A5000BE1BB1400D43691E8D4100212C43BCE685
:107A6000802100260903134C0025BBE50D43691E48
:107A70008D410021EDB269E7010015000D4C1AE5BA
:107A80000100150017E51C000F00203CE7403C00FA
:107A9000202B0CD04027FB1A99400D43691E8D41C5
:107AA0000021254352E70021D4E71D0092E5002183
:107AB000F3E7C046FF070000FFFF7FFFF0B55F461A
:107AC00056464D464446F0B41F035C00DB0F9A4611
:107AD000194B0E034D00C90F8046360B6D0D8B46BA
:107AE00091463F0B640D9D4219D0134B9C421BD015
:107AF0000123A54206D018003CBC90469946A246F8
:107B0000AB46F0BDBE42F6D1C845F4D1D34510D046
:107B1000002DF0D1304303005A1E9341EBE73100B2
:107B200001230143E7D1E0E73A430123002AE2D1F0
:107B3000DEE70023DFE7C046FF070000F0B55F4641
:107B4000444656464D46F0B41F033C0B2C4F0E03E3
:107B50004D00A3465C008446360B6D0DC90F904660
:107B6000640DDB0FBD422BD0254FBC422ED0002D23
:107B70000ED130430700814678427841002C17D15E
:107B80005F463A4314D14B460020002B0AD006E052
:107B9000002C02D15846024301D099421AD0012349
:107BA000484218433CBC90469946A246AB46F0BDBD
:107BB0000028F2D058425841012240421043F1E7D8
:107BC00037000743D0D002204042EBE75F4617431F
:107BD000CDD0F8E7A542E2DC05DB5E45DFD808D072
:107BE00000205E45DED2484248410123404218430E
:107BF000D8E7C445D3D80020C445F4D3D2E7C04663
:107C0000FF070000F0B55F464D4644465646F0B4C7
:107C10001C03240BA4462F4C0F034D005E00C90F1C
:107C200080463F0B6D0D8B469146760DDB0FA542CE
:107C300020D0284CA64222D0002D12D138434442F5
:107C40004441002E20D0002C0DD05C426341012421
:107C50005B421C4320003CBC90469946A246AB4682
:107C6000F0BD002E17D05B4519D05B465C42012366
:107C70001C43EFE7390002240143EBD1D9E7614609
:107C800002241143E6D1D7E761460A43DBD1002441
:107C90000028DFD0E9E761460A43E4D1E5E7B542D1
:107CA00003DD01225C421443D4E7B542CDDB6745D6
:107CB000DBD809D000246745CCD259464C426141FB
:107CC000012449420C43C5E7C845CED80024C84525
:107CD000F3D3BFE7FF070000F0B55F4656464D46B9
:107CE0004446F0B40D0399464E002B0B87B00700B5
:107CF000924680469B46760DCC0F002E69D06D4B88
:107D00009E4235D05B468022DD001204430F1343B0
:107D10002B439B46C3009846674B00279C46002395
:107D2000664401934A4615035000D20F53462D0B6B
:107D3000400D914600D176E05E4A90426CD08022A0
:107D40005B0F120413435C4AED0094461D435346F7
:107D50000022DB00604449463618701C61400290E6
:107D600017430F2F00D9AFE05448BF00C759BF4693
:107D70005B461F4300D088E000239B4698460233B1
:107D800008270193CEE74946022A6AD0032A00D188
:107D900009E2012A00D0BBE11140002200230025A6
:107DA0009046CCB200212D030A0D12052D0B154370
:107DB000434A1B0515401D436D00E4076D0825432C
:107DC0004046290007B03CBC90469946A246AB46C7
:107DD000F0BD034352D05B46002B00D18AE15846E8
:107DE00000F014FE03000B3B1C2B00DD7BE11D2289
:107DF000D31A3A0001005D46DA4008398D4013007D
:107E00008F402B439B46B8462E4B00279C460023B1
:107E100060444642019385E752462A432CD100250F
:107E20000023022297E752462A4321D0002D00D199
:107E300054E1280000F0EAFD03000B3B1C2B00DDA1
:107E400046E11D21CB1A51460200D9405346083A5B
:107E5000954093400D431B4A9446604440420022A3
:107E600079E7012400220C40124B0025904699E747
:107E70000025002301226EE703226CE700239B46C6
:107E800098460133042701934CE703230C27019301
:107E900048E700238025984600242D03054B81E701
:107EA0005D464346019A6FE75D4643462100019ACD
:107EB0006AE7C046FF07000001FCFFFF50AF00006B
:107EC000FFFF0F80F30300004246120C91461A0C8C
:107ED0009446424617044A461B041B0C5A4360460C
:107EE00090464A4642431000039262461C003F0CF3
:107EF0007A437C4342440192220C9246019A5244B6
:107F0000904506D98246802040028046C2445046B1
:107F10000390100C049048462404240C12041219F7
:107F200005922A0C2D042D0C68432C0082464846ED
:107F30007C4350438146200C804657435744474476
:107F4000BA4503D9802040028046C144380C3F0422
:107F5000B84648442404240C01900498A0444044AA
:107F600004905846000C814658460404200C824672
:107F7000070048465F434C464343604660436446BF
:107F8000834650464443380C8446E4186444A34274
:107F900003D980235B029C46E34448463F04230CFC
:107FA0003F0C2404E419574668436F4384464D460A
:107FB000504655434243380C814662444A445B4430
:107FC000944503D9802040028446654403983F04C9
:107FD000834604983F0C8446E344C34580414042B5
:107FE0008246100484460198674484466744A3444B
:107FF000BC46A345A4419946D44464428742BF414C
:10800000D4458041E144A04699459B417F4240428E
:10801000C8440743120CBA18A045A4415F423B0074
:1080200064422343D71843467D19DB0D6D021D437F
:108030005B465A02059B1A43531E9A415B46DB0D71
:108040001A4343465B021343EA0107D501225C0849
:1080500013402343EA07029E13436D08574AB218A0
:10806000002A4BDD580709D00F201840042805D0FE
:10807000181D98429B415B42ED180300E80104D5AE
:108080004F4A15408022D200B2184E48824200DD8D
:10809000E7E60124DB08680718436D0253058046B4
:1080A0002D0B5B0D0C407DE68022594612031142D8
:1080B00008D0154206D115432D0398462D0B4C468A
:1080C000414B6FE65D4615432D032D0B3E4B69E694
:1080D00003005546283B9D400023BCE6504600F077
:1080E00095FC2030A8E60300283B9F400023BB46B8
:1080F000984689E600F08AFC203073E60124A61A2F
:10810000382E07DD00220C4000230025904649E66A
:10811000029EA3E71F2E20DC20222C001800921BB9
:10812000F040944093400443581E83411C43F54063
:10813000630709D00F232340042B05D023001C1D07
:108140009C4292415242AD182B021FD501240022BD
:108150000C4001230025904624E61F202C004042BD
:10816000821AD440202E1CD04022961BB5402B43AF
:10817000581E83410720234318400025002809D0BA
:108180000F2200251A401C00042AD8D123006807BA
:108190006D022D0B0124DB08034398460C4000239D
:1081A00000E60025E3E780220124120315432D0396
:1081B00098462D0B0C40044BF4E5C046FF0300002D
:1081C000FFFFFFFEFE070000FF070000F0B5574667
:1081D0004E464546E0B40E001100F20F9246C5002F
:1081E000420F180337037400400A4E0F7F0A3043D2
:1081F000CF4E17435A00640D520DDB0FC900B24237
:1082000000D1E5E001267340A61AB446534500D1DB
:10821000AFE0002E00DC0DE1002A3AD103000B4351
:1082200000D0E4E06B0709D00F232B40042B05D0CE
:108230002B1DAB42AD416D427F191D003B0200D4A6
:1082400088E0BB4B01349C4200D110E13A00B94BAD
:1082500051461A4001235007ED08520264050543B8
:10826000120B640D0B400021280012030D0D120BA0
:1082700064052D0515436208AF4CDB072C40144301
:10828000640064081C4321001CBC90469946A24629
:10829000F0BDA74B9C42C5D080231B041843634606
:1082A000382B00DDFDE01F2B00DD30E1624620238E
:1082B0009B1A02009A40664690460A009940F24096
:1082C00046464B1E99413243114363460200DA4051
:1082D000691A8D429B410D00BA1A5B42D71A3B02C4
:1082E00035D57A02530A98464346002B00D1C4E0A4
:1082F000404600F08BFB0300083B1F2B00DDC5E070
:1083000020222900D21A4746D1409F400A009D40B2
:108310003A439C4200DDC0E01C1B631C1F2B00DDA8
:10832000E4E0202114002800C91AD8408C408D4078
:108330000443DA40681E854117002543002471E795
:10834000424663461A4300D14CE2674645466B07F6
:1083500000D069E7012351467807ED08FA080B4081
:10836000054373498C4238D012036405120B640D27
:1083700079E7002E00DC9AE0002A47D06C4A94424C
:1083800000D14FE78022120410436246382A00DCF5
:1083900008E10143481E81410022C9B24919D2199E
:1083A000A942BF410D007F42BF183A0200D442E10A
:1083B0005F4A0134944200D14EE101205D4A6908D0
:1083C0003A4028400843D507054357089A4629E70D
:1083D00006000E4300D017E714E72900114300D12F
:1083E000F9E1802109030A431203120B3BE7012341
:1083F0005B429846C4446346002B72D1691A8D4291
:108400009B413F1A5B42FF1A0D0068E702000A43D6
:1084100000D107E7012252429046C4446246002A36
:1084200000D0E6E06918A942B6413F187642F71934
:108430000D00BAE7002E00D080E0621C5205520DFC
:10844000012A00DCF9E06A1A91464D45B6413A1A14
:108450007642921B9046120200D499E04D1BA9422D
:108460008941C71B49427A1A90469A463CE75246D0
:108470000123002513400022F5E6280000F0C6FA8B
:1084800020300300083B1F2B00DC39E72A00283886
:10849000824000259C4200DC3EE7264FE41A17404C
:1084A000C0E60143481E81410022C9B210E7002EF8
:1084B00000D0F1E0621C94465205520D012A00DC06
:1084C000A0E01B4A944500D1C5E06918A942924139
:1084D0003F185242D2194908D5070D435708644640
:1084E000A0E6134B9C4200D0D9E69BE611001F3C4E
:1084F000E1400C00202B00D180E04021CB1A9A40B3
:1085000015436A1E95410027254300241FE7634653
:108510000200203BDA406346202B71D040236646A0
:108520009B1B98400143481E814111430022CFE626
:10853000FF070000FFFF7FFFFFFF0F80002C48D0E8
:10854000CA4CA24200D1A2E07442A1468024240475
:1085500027434C46382C00DDDBE01F2C00DD44E1D6
:108560004E462024A41B3E00A640A246B0464C46E0
:108570002E00E640B4464646644626435446A5408F
:108580006C1EA54134002C434D46EF400D1B28E0E6
:108590004A4643464D461A4300D0A5E60023002430
:1085A0000025DEE61F2A5ADC66462022921B0600C2
:1085B00096409146B04662460E00D640424616436B
:1085C0004A4691404A1E9141020060463143C240F2
:1085D000E4E63C002C435AD0F443A146002C52D18F
:1085E0004D1BA9428941C71B49427F1A14009A4674
:1085F00075E69E4A944200D0C7E613E600227FE764
:1086000000208FE7002C00D0C8E03B002B4300D1B6
:108610000FE103000B4300D104E66918A9429B4116
:108620003F185B42DF193B0200D41AE1904B0D006A
:108630001F406446F6E59A4689E63A002A43002C34
:108640005CD1002A75D102000A4300D1CAE00700BC
:108650000D009A46E6E564460022002581E6624662
:108660000600203AD6406246B046202A00D1B7E044
:1086700040226646921B904001434246481E81417B
:10868000114300228AE6794CA24200D061E707003C
:108690000D0014009A46C5E5002C41D13C002C4346
:1086A00078D0F443A146002C20D0704CA24271D067
:1086B0004C46382C00DDB2E01F2C00DDBCE020264B
:1086C000341BA2463C005646B4404E46A0462C0001
:1086D000F440A446444666463443A4465446A54066
:1086E00064466E1EB54125434C46E7406D188D42E9
:1086F00089413F184942CF19140056E6002A2FD16C
:1087000002000A4300D184E007000D009A46574C4E
:1087100088E53D436F1EBD41ECB200270D1B60E7AD
:10872000524CA24236D0744280263604A1463743CA
:10873000BEE702000A4300D174E56A1A9046454537
:10874000B6413A1A7642921B9446120200D4F7E5DB
:108750004D1BA9428941C71B49427F1A9A4661E5D0
:1087600002000A433AD0ED087C072C438025FA0822
:108770002D032A4208D0C7082F4205D145072C00F7
:108780003A009A46C9080C43670FD200E500174328
:10879000364C47E507000D00140043E53A002A4334
:1087A00043D002000A4319D0ED087C072C438025F2
:1087B000FA082D032A4207D0C6082E4204D14707E3
:1087C0003C003200C9080C43D700620FE500174394
:1087D0009A46264C26E50022002544E5234C21E557
:1087E000002049E700230025BBE54C463E00203C25
:1087F000E6404C46B446202C31D040244E46A61BC1
:10880000B7403D436C1EA54164462C4300270D1B19
:10881000E7E6802200231203144C0025A1E53D4326
:108820006F1EBD410027EDB260E707000D000F4C41
:10883000F8E407000D00F5E44E463C00203EF4400D
:10884000A0464C46202C0ED040244E46A41BA740E8
:108850003D436F1EBD4144460027254346E70027A0
:10886000CFE70D0073E50027F2E7C046FF070000E1
:10887000FFFF7FFF0B0330B5134D1A0B4B005B0D51
:10888000C90F0024AB4211DD104CA34210DC802440
:10889000640322430E4CE41A1F2C0CDD0D48C31A4E
:1088A000DA4013005C42002900D11C00200030BDDA
:1088B000094BCC18FAE7E040084CA44663449A40C0
:1088C00013000343EEE7C046FE0300001D04000052
:1088D0003304000013040000FFFFFF7FEDFBFFFFE8
:1088E00070B5002830D0C317C4185C40C50F2000F5
:1088F00000F08CF8174B184A1B1AD21A1F2A18DDE1
:10890000164AD21A9440002224035B05240B5B0D07
:108910000021100024030A0D1205240B1443104AF1
:108920001B0514401C436400ED0764082C43210020
:1089300070BD210091400A000B21081AC4405B055C
:108940002403240B5B0DE3E7002500230024002211
:10895000DEE7C0461E0400003304000013040000DC
:10896000FFFF0F804200120E511C4302C9B270B5C6
:108970005D0AC40F012915DDE02189008C466D07D1
:108980001B0B6244002128000D0D2D052B431C4DAF
:1089900052052B40520813435B00E4075B08234356
:1089A000190070BD002A15D1002D1FD0280000F03D
:1089B0002DF80A281DDC0B232A001B1ADA401300AD
:1089C0000200153295400F4A1B03121A52051B0B69
:1089D000520DD7E7002D06D080221B0B1203134344
:1089E0006D07094ACEE7084A0023CBE7002200239F
:1089F000C8E703000B3B9D402B000025E3E7C04682
:108A0000FFFF0F8089030000FF0700001C210123E6
:108A10001B04984201D3000C10391B0A984201D361
:108A2000000A08391B09984201D30009043902A23F
:108A3000105C40187047C0460403020201010101A6
:108A400000000000000000007FB51D000A4B06007A
:108A50001B68D868002A02D1084C230001E01300EB
:108A6000074C0293009133002A000649019400F05C
:108A700021F800F023FEC0468C02002016A9000059
:108A800090AF00009DAF0000084B10B50400002B14
:108A900002D0002100E000BF054B1868836A002B5C
:108AA00000D09847200001F0F3FAC0460000000013
:108AB000D0AF00000EB403B5010003AB044804CBF3
:108AC0000068019300F016F902B008BC03B0184723
:108AD0008C0200200E4B70B500251E000D4CE41AD0
:108AE000A410A54204D0AB00F35898470135F8E72D
:108AF00001F0D0FA084B00251E00084CE41AA4101F
:108B0000A54204D0AB00F35898470135F8E770BD93
:108B1000940200209402002094020020A40200206D
:108B200010B5034B0100186800F066F810BDC04690
:108B30008C02002010B5034B0100186800F016F8F5
:108B400010BDC0468C020020002310B59A4203D00D
:108B5000CC5CC4540133F9E710BD03008218934282
:108B600002D019700133FAE77047000030B50029D0
:108B70003ED004390B68002B00DAC9181D4A13686F
:108B80001400002B02D14B60116031E08B420DD9F3
:108B90000A688818834203D118685B6882180A60E3
:108BA0004B60216024E08A4203D813005A68002AEF
:108BB000F9D11D685C198C420BD1096869185818E5
:108BC0001960824214D110685268411819605A60C5
:108BD0000EE08C4202D90C23036009E008680C18EF
:108BE000A24203D114685268201808604A60596094
:108BF00030BDC04664120020032370B5CD1C9D43D8
:108C0000083506000C2D01D20C2505E0002D03DAF5
:108C10000C230020336040E0A942F9D81F4B1C68A8
:108C20001A002100002913D00B685B1B0DD40B2BFD
:108C300002D90B60CC181EE08C4202D1636813602D
:108C40001AE04B6863600C0016E00C004968E9E725
:108C5000134C2368002B03D1300000F033FB20605D
:108C60002900300000F02EFB431CD1D00323C41C8C
:108C70009C43A0420AD12560200007220B30231D0F
:108C80009043C31A09D05A42E25006E0211A30003C
:108C900000F018FB431CEED1BAE770BD641200204F
:108CA00060120020936810B5013B9360002B05DA39
:108CB0009469A34208DBCBB20A2B05D01368581C79
:108CC00010601970C8B201E000F02CFC10BDF8B5BE
:108CD00006000F001400D518AC4208D021783A00E5
:108CE0003000FFF7DFFF0134431CF5D100E0002026
:108CF000F8BD0000F0B59FB006000F00029205938A
:108D0000002804D08369002B01D100F0D3FD7F4BF4
:108D10009F4201D1776808E07D4B9F4201D1B7683F
:108D200003E07C4B9F4200D1F768BB891B070AD543
:108D30003B69002B07D0002306AD6B6120336B76B7
:108D40001033AB763DE03900300000F043FC0028E2
:108D5000F1D001204042D6E0059A111D126805911C
:108D6000002A00DA7FE00992013423782E2B00D10B
:108D70008DE021780322684800F082FE002807D0A9
:108D8000654B2A68C01A4023834013432B6001348B
:108D90002178631C062261480293297600F070FE58
:108DA000002800D19DE05E4B002B00D090E0072210
:108DB000059B07339343083305936B69039A9B180C
:108DC0006B61029C2378002B04D1029BE31A04936D
:108DD00012D003E0252BF8D00134F3E7049B029A6C
:108DE00039003000FFF773FF431C00D186E06A6949
:108DF000049B944663446B612378002B7ED0012250
:108E0000002352426A6002A95432521801342B6086
:108E1000EB60AB601370AB6521780522414800F030
:108E20002FFE002808D03F4B2A68C01A0123834038
:108E300013432B600134EFE72B68DA0604D5532285
:108E4000202102A8121811701A0704D553222B21D1
:108E500002A81218117022782A2A00D17CE7099BF7
:108E600000200A2105E05242EA60022213432B60EF
:108E70007AE72278303A092A04D84B4301349B1808
:108E80000120F6E7002800D16FE709936DE76378CA
:108E90002A2B0AD1059B02341A1D1B680592002B50
:108EA00001DA01235B42079363E700230A201A00DB
:108EB00001346B6021783039092904D842430134E8
:108EC00052180123F6E7002B00D152E7079250E732
:108ED00005AB00933A00144B2900300000E000BFBE
:108EE00007E005AB00933A000F4B2900300000F07B
:108EF0008BF80390039B013300D05EE7BB895B06D0
:108F000000D526E70B981FB0F0BDC04608B10000A1
:108F100028B1000048B10000DAAF0000DEAF000069
:108F200000000000D4AF0000CF8C0000F7B51700A0
:108F300001938A680B6900900C00934200DA1300D9
:108F400022003B6043321278002A01D001333B609B
:108F500023689B0602D53B6802333B6006252368E5
:108F60001D401ED0230043331B785A1E93412268B4
:108F700092061CD53020E1184331087021005A1C9C
:108F800045310978A2184332023311700FE02200F4
:108F90000123193201990098089EB047431C0ED056
:108FA0000135E3683A689B1A9D42F0DBDAE722005C
:108FB000019943320098089DA847431C02D1012023
:108FC000404220E006232068E1683A68034000251B
:108FD000042B03D18D1AEB43DB171D40A3682269D4
:108FE000934201DD9B1AED180027BD420AD02200F2
:108FF00001231A3201990098089EB047431CDED025
:109000000137F2E70020FEBDF0B58BB006920A00F2
:1090100043320793059004920A7E0C00109B6E2A3F
:1090200000D1ABE011D8632A22D009D8002A00D1A0
:10903000B5E0582A00D0C5E045310A70814A4FE0BA
:10904000642A1DD0692A1BD0BCE0732A00D1AAE093
:1090500009D86F2A29D0702A00D0B3E020220968ED
:109060000A43226037E0752A1FD0782A33D0A9E05E
:109070000E001A684236111D196013683370A4E09F
:1090800021681A68080606D4490604D5111D19601E
:109090000023D55E02E0111D19601568002D3BDA32
:1090A0002D23049A6D42137036E021681A68080671
:1090B00006D4490604D51568111D1960ADB202E049
:1090C000111D196015685F4B227E039308276F2AD4
:1090D0001DD00A271BE022007821453211705A4A20
:1090E00019680392081D226818600D68100602D4E2
:1090F000500600D5ADB2D30702D520231A43226013
:109100001027002D03D1202322689A4322602300D8
:10911000002243331A7002E00A274A4B0393636824
:10912000A360002B09DB0422216891432160002DFC
:1091300005D1049E002B11D07BE0002D79D0049E38
:1091400028003900FDF7CAFE039B013E5B5C280046
:1091500033703900FDF73CFE051EF1D1082F09D10F
:109160002368DB0706D563682269934202DC30235B
:10917000013E3370049B9B1B23612BE009681A6836
:10918000080607D4490605D5111D19601368A28A7F
:109190001A8004E0111D1960136862691A600023C7
:1091A000049E236116E01A68111D196016680021DB
:1091B0006268300000F064FC002801D0801B606011
:1091C000636803E0260042363270012323610023E6
:1091D000049A1370079B09AA00932100069B059827
:1091E000FFF7A4FE431C02D10120404227E023697F
:1091F000320006990598079DA847431CF4D02368C0
:1092000000259B070FD4099BE068984217DA1800E5
:1092100015E022000123193206990598079EB047F0
:10922000431CE1D00135E368099A9B1A9D42F0DBAB
:10923000E9E72600039B42361B7833708EE70BB0BC
:10924000F0BDC046E5AF0000F6AF0000154B10B50D
:109250001C68A36B002B15D11820FFF761FC124B83
:10926000A0630380114B01224380114B8380114B7B
:10927000C380114B0381052343810633838100237F
:1092800002614361A46B0D4A206961690C4BFDF7D3
:1092900061FF01220023801859412061616148006B
:1092A000400810BD8C0200200E330000CDABFFFF44
:1092B000341200006DE6FFFFECDEFFFF2D7F954CC2
:1092C0002DF45158002370B5064C050008002360AA
:1092D00000F0C8FE431C03D12368002B00D02B6094
:1092E00070BDC0467C2600200CB430B5164B9DB036
:1092F0000C1E1D6804DA8B2301202B6040421DE008
:10930000822302A99B008B810023029008619C426A
:1093100000D0631E8B604B6101235B42CB81209A9E
:1093200021AB2800019300F053FC431C01DA8B238E
:109330002B60002C02D00023029A13701DB030BCA9
:1093400008BC02B01847C0468C0200200EB410B50D
:109350009DB002A9029008610B4882248860486190
:10936000012040421FABC881084804CBA40000681C
:1093700001938C8100F02CFC0023029A13701DB025
:1093800010BC08BC03B01847FFFFFF7F8C02002011
:1093900002780B78002A03D0013001319A42F7D0CD
:1093A000D01A7047031C0A7801311A700133002A61
:1093B000F9D170470023C25C0133002AFBD1581E4B
:1093C0007047030030B5002A0DD00C7801335D1EC4
:1093D000013A2C700131002CF5D19A189A4202D032
:1093E0001C700133FAE730BDF0B51E00454B87B065
:1093F0001B680192029308220B00059003911C78D0
:1094000002995D1C09194878104001D02B00F6E73D
:109410002D2C04D19D1C5C780123009304E0009066
:109420002B2C01D15C789D1C002E02D0102E0AD16D
:1094300062E0302C5ED120222B789343582B54D1FC
:1094400010266C780235009F31007B1E9F412E4B09
:10945000FF183800FDF742FD380004913100FDF798
:10946000B7FC00230322070094461800029A121941
:1094700051780422114201D0303C07E0624611408D
:1094800017D03722012900D02032A41AA64210DDBD
:109490005A1C0BD0B84207D802D1049B9C4203DC73
:1094A00070430123201801E001235B422C78013531
:1094B000DCE75A1C0BD10098059A431E9841124BC9
:1094C000C01822231360019B002B0AD117E0009AD9
:1094D000002A00D04042019A002A10D0039A002BA3
:1094E00000D06A1E019B1A6009E03024002EAAD128
:1094F0000826A8E70A26A6E7302C9CD0A3E707B0E9
:10950000F0BDC04690020020FFFFFF7F10B51300A2
:109510000A00010002480068FFF766FF10BDC04660
:109520008C020020F8B505000F001400002804D0BC
:109530008369002B01D100F0BDF9234B9C4201D17E
:109540006C6808E0214B9C4201D1AC6803E0204BE1
:109550009C4200D1EC68A369A360A3891B070AD5CC
:109560002369002B07D023682269FEB2981A636929
:1095700098420FDB08E02100280000F02BF80028BB
:10958000F1D0012040421DE02100280000F024F924
:109590000028F6D1A3680130013BA36023685A1C60
:1095A00022601F706369984205D0A3893000DB07F1
:1095B00008D50A2E06D12100280000F00DF9002858
:1095C000DFD13000F8BDC04608B1000028B100006E
:1095D00048B10000354B70B51D6806000C00002D29
:1095E00005D0AB69002B02D1280000F063F9304BA5
:1095F0009C4201D16C6808E02E4B9C4201D1AC68C2
:1096000003E02D4B9C4200D1EC68A3899AB211076C
:1096100023D4D10607D40922012032603732134304
:10962000A381404240E0530713D5616B002908D065
:1096300023004433994202D03000FFF797FA002309
:1096400063632422A3899343A38100236360236976
:1096500023600822A3891343A3812369002B0BD124
:10966000A023A2899B00134080229200934203D042
:109670002100300000F0B2F90123A289134005D087
:109680000023A36063695B42A36103E0910700D4F8
:109690006369A36000202369834205D1130603D5C3
:1096A00040231A43A281013870BDC0468C020020BD
:1096B00008B1000028B1000048B1000010B5062034
:1096C00000F0AEFB012000F0E3FC0000F7B58A8952
:1096D00005000C0013075AD44B68002B02DC0B6CFE
:1096E000002B19DDE76A002F16D000232E682B60AF
:1096F00080235B011A4001D0606D14E00123216AD0
:109700002800B847431C0ED12B68002B0BD01D2B13
:1097100001D0162B02D12E6000205AE04022A389EE
:109720001343A38155E0A3895B0706D56368C01A7C
:10973000636B002B01D0236CC01A00230200216A46
:109740002800E76AB847A389421C06D129681D2969
:109750003AD8204ACA40D20736D500226260226930
:109760002260DB0405D5431C02D12B68002B00D1FD
:109770006065616B2E600029CED02300443399428E
:1097800002D02800FFF7F2F90020606321E00F69A2
:10979000002FC1D00B680F60DB1B019300239207E1
:1097A00000D14B69A36003E0019B3F181B1A019392
:1097B000019B002BB0DD019B3A00216A2800A66ABC
:1097C000B0470028F0DCA389402201201343A38185
:1097D0004042FEBD010040200B6970B505000C0041
:1097E000002B01D100201CE0002804D08369002B4D
:1097F00001D100F05FF80B4B9C4201D16C6808E08E
:10980000094B9C4201D1AC6803E0084B9C4200D15B
:10981000EC680C22A35E002BE4D021002800FFF7A7
:1098200055FF70BD08B1000028B1000048B100002C
:1098300010B5024900F0B0F810BDC046D99700003D
:10984000002310B504000360436083608181436698
:10985000C281036143618361190008225C30FFF714
:109860007CF9054B24626362044BA362044BE36200
:10987000044B236310BDC046619E0000899E00001A
:10988000C19E0000ED9E000070B568254B1E5D4333
:109890000E0029007431FFF7AFF9041E08D0002133
:1098A0002A00016046600C30A0606832FFF755F96D
:1098B000200070BD836913B50400002B28D1836498
:1098C000C3640365134B144A1B6882620193984278
:1098D00001D101238361200000F020F860602000A6
:1098E00000F01CF8A060200000F018F80022E060F2
:1098F00004216068FFF7A4FF01220921A068FFF797
:109900009FFF02221221E068FFF79AFF0123A36163
:1099100013BDC046D0AF000031980000F8B51D4B14
:1099200006001D68AB69002B02D12800FFF7C2FFBB
:109930004835AC686B68013B05D40C22A75E002F4C
:1099400010D06834F7E72B68002B01D02D68F0E7C2
:1099500004213000FFF798FF28600028F6D10C237F
:10996000336016E0012320005B42E3810233A381D0
:1099700067662760A760676027616761A7615C30E1
:1099800008223900FFF7E9F820006763A763A7649E
:10999000E764F8BDD0AF0000F7B50400070000266B
:1099A00001914834002C16D06368A5680093009B91
:1099B000013B00930DD4AB89012B08D90E22AB5E7D
:1099C000013304D029003800019B984706436835CD
:1099D000EDE72468E6E73000FEBD0000F0B58B89B6
:1099E00091B006000C009B0726D40E23C95E002907
:1099F00004DA8023A5891D4010D10CE001AA00F0F3
:109A0000A1FA0028F5DBF023029D1B021D401A4B32
:109A1000ED186B425D418027FF0001E000254027E3
:109A200039003000FFF7E8F800280CD1A3899A0527
:109A30001FD402221343A3812300473323602361F1
:109A40000123636115E080220C4BB362A38920607F
:109A50001343A38120616761002D0AD00E23E15ECC
:109A6000300000F081FA002803D00122A3891343BB
:109A7000A38111B0F0BDC04600E0FFFF31980000A7
:109A8000C9B28218904204D003788B4202D00130D0
:109A9000F8E70020704710B5884202D98B18984229
:109AA00001D3002305E09B1A013A08D3995C815445
:109AB000FAE7934203D0CC5CC4540133F9E710BDFC
:109AC000F8B506000C001500002904D11100FFF7BD
:109AD00093F8040018E0002A03D1FFF747F82C00A0
:109AE00012E000F067FA85420ED929003000FFF736
:109AF00083F8071E07D021002A00FFF725F8210070
:109B00003000FFF733F83C002000F8BDF0B58E6858
:109B100085B007000C00039201939E4243D8902326
:109B20008A89DB001A423ED003250969236801981F
:109B30005B1A029363695D43EB0F5D19029B6D1025
:109B400001331B18AB4200D91D00530510D5290065
:109B50003800FFF751F8061E14D0029A2169FEF76B
:109B6000F3FFA289194B134080221343A38112E013
:109B70002A003800FFF7A4FF061E0CD12169380027
:109B8000FEF7F4FF0C23402201203B60A3894042F2
:109B90001343A38117E0029B2661F61826606561D6
:109BA000019EED1AA560019BB34200D21E00320057
:109BB00003992068FFF76FFF0020A3689B1BA36039
:109BC00023689E19266005B0F0BDC0467FFBFFFFED
:109BD000F0B59FB0029005938B890F0016001B060D
:109BE00010D50B69002B0DD14021FFF705F8386027
:109BF0003861002804D10C23029A01381360D8E0A0
:109C000040237B61002306AD6B6120336B761033FC
:109C1000AB7634002378002B03D1A31B049312D01E
:109C200003E0252BF9D00134F4E7A31B32003900FF
:109C30000298FFF76BFF431C00D1B4E06A69049BF4
:109C4000944663446B612378002B00D1ABE0012282
:109C5000002352426A6002A95432521801342B6028
:109C6000EB60AB601370AB65534E2178052230007A
:109C7000FFF706FF002807D00123801B83402A68D6
:109C8000013413432B60EFE72B68DA0604D5532227
:109C9000202102A8121811701A0704D553222B2173
:109CA00002A81218117022782A2A03D0099B0020DA
:109CB0000A210EE0059A111D12680591002A01DBA8
:109CC000099204E05242EA60022213432B600134FD
:109CD0000BE02278303A092A04D84B4301349B1810
:109CE0000120F6E7002800D0099323782E2B1ED1FF
:109CF00063782A2B0AD1059B02341A1D1B68059232
:109D0000002B01DA01235B42079310E000230A20B5
:109D10001A0001346B6021783039092904D8424394
:109D2000013452180123F6E7002B00D00792234E8E
:109D3000217803223000FFF7A3FE002806D040233D
:109D4000801B83402A68013413432B60217806224C
:109D50001B48661C2976FFF793FE002812D0194B8A
:109D6000002B06D10722059B073393430833059345
:109D700014E005AB00933A00134B2900029800E071
:109D800000BF07E005AB00933A000F4B2900029893
:109D9000FFF73AF90390039B013304D06B69039AF0
:109DA0009B186B6135E7BB890B985B0601D50120D9
:109DB00040421FB0F0BDC046D4AF0000DAAF000093
:109DC000DEAF0000000000000D9B000070B5040035
:109DD0000D1E1F2D04D916230360012040421EE0F2
:109DE000426C002A04D08B00D2181368002B08D1D3
:109DF000200000F031F82A000100200000F01AF8DD
:109E00000DE00020012B0AD0591C03D11733236029
:109E1000013004E00024280014609847200070BD41
:109E200010B5034B01001868FFF7D0FF10BDC04606
:109E30008C020020002370B5064C050008001100BC
:109E4000236000F0F7F8431C03D12368002B00D0F7
:109E50002B6070BD7C26002010B500F0DBF810BD33
:109E600070B50C000E25495F00F0B0F8002803DB48
:109E7000636D1B18636503E0A289024B1340A38145
:109E800070BDC046FFEFFFFFF8B51F008B890500CE
:109E90000C001600DB0505D50E23C95E0022022347
:109EA00000F074F8A289054B28001340A38132000A
:109EB0000E23E15E3B0000F01FF8F8BDFFEFFFFF4F
:109EC00070B50C000E25495F00F060F8A389421CB4
:109ED00003D1054A1340A38104E0802252011343B9
:109EE000A381606570BDC046FFEFFFFF10B50E2374
:109EF000C95E00F015F810BD70B50500080011002E
:109F00000022064C22601A0000F0BAF8431C03D16C
:109F10002368002B00D02B6070BDC0467C2600203B
:109F2000002370B5064C05000800236000F062F8BD
:109F3000431C03D12368002B00D02B6070BDC046AA
:109F40007C260020002370B5064C05000800110097
:109F5000236000F057F8431C03D12368002B00D086
:109F60002B6070BD7C260020002370B5064C0500D8
:109F70000800236000F056F8431C03D12368002B2F
:109F800000D02B6070BDC0467C26002070B5050057
:109F9000080011000022064C22601A0000F052F85E
:109FA000431C03D12368002B00D02B6070BDC0463A
:109FB0007C2600200B1F1A68101F002A04DA89185B
:109FC00004390B68D01804387047000070B50500DC
:109FD000080011000022064C22601A0000F03AF836
:109FE000431C03D12368002B00D02B6070BDC046FA
:109FF0007C26002058220120014B40421A60704705
:10A000007C26002058220120014B40421A607047F4
:10A010007C26002058220120014B40421A607047E4
:10A020007C2600205822024B00201A607047C04650
:10A030007C26002058220120014B40421A607047C4
:10A040007C26002058220120014B40421A607047B4
:10A050007C26002058220120014B40421A607047A4
:10A060007C260020044A1368002B03D018181060C7
:10A0700018007047014BF9E7681200208026002085
:10A0800058220120014B40421A6070477C26002074
:10A09000FEE7C046F8B5C046F8BC08BC9E4670470F
:10A0A000F8B5C046F8BC08BC9E46704766616C7344
:10A0B000650074727565006C697374206F66202585
:10A0C00064206974656D73006F626A656374206FE4
:10A0D0006620636C6173733A202564005374616376
:10A0E0006B20756E646572666C6F770036060000D3
:10A0F000C8050000460600007C060000B806000007
:10A10000F20600002E07000056070000940700002A
:10A11000DA070000360800007C080000EA080000AA
:10A1200038090000600900009A090000E4090000F5
:10A130000C0A0000440A00007E0A0000BA0A00006F
:10A14000400B0000080C0000980C0000F60C00000A
:10A15000400D0000620D00006A0D00004C0E000072
:10A16000980E000036060000360600003606000095
:10A17000140F00007E0F0000001000004A100000C5
:10A18000981000001E110000A6110000F41100003C
:10A190003E12000074120000C01200000C130000F8
:10A1A00060130000BC1300001814000056140000D7
:10A1B000C2140000FA1400004615000092150000B9
:10A1C000DE1500001816000064160000B01600002E
:10A1D0003606000036060000360600002017000094
:10A1E0005817000090170000BE170000F617000077
:10A1F000241800003606000036060000360600006F
:10A20000360600005C180000A418000036060000A6
:10A2100036060000F01800001E1900006819000042
:10A2200036060000360600003606000096190000CB
:10A23000C6190000F6190000261A0000521A000084
:10A240008A1A0000B61A0000F81A0000221B00004B
:10A25000521B0000821B0000AE1B0000DA1B000036
:10A260000A1C0000361C00003606000036060000FE
:10A27000360600003606000036060000661C0000A8
:10A28000941C0000C21C0000F01C00001E1D0000F9
:10A29000561D00008E1D0000C61D0000FE1D0000A2
:10A2A0002C1E00005A1E00009C1E000036060000F6
:10A2B00036060000360600003606000036060000AE
:10A2C000360600003606000036060000360600009E
:10A2D000360600003606000036060000360600008E
:10A2E00036060000CA1E0000F81E0000070000002D
:10A2F000030000006D6963726F3A626974006861FF
:10A3000073546F6E6500706C6179546F6E65006890
:10A310006173536572766F00736574536572766FFF
:10A32000000000000000000001000000020000002A
:10A3300003000000040000000A0000000D0A564D52
:10A340002050616E69633A2025730D0A00496E73CF
:10A35000756666696369656E74206D656D6F727987
:10A3600020666F72204D6963726F426C6F636B730E
:10A37000206F626A656374206865617000496E735E
:10A38000756666696369656E74206D656D6F727957
:10A3900020666F72204D6963726F426C6F636B73DE
:10A3A00020737461636B00626164206F626A65632D
:10A3B0007420617420256C640A0025783A20256495
:10A3C00020776F7264732C20636C6173734944202F
:10A3D00025640A004865616465723A2025780A00A0
:10A3E00009307825782C0A006D69736300686578F8
:10A3F000546F496E740073696E006E657400686115
:10A4000073576946690073746172745769466900CD
:10A4100073746F7057694669007769666953746130
:10A42000747573006D79495041646472657373008B
:10A430007468696E674465736372697074696F6E7E
:10A4400000636C6561725468696E6744657363721A
:10A45000697074696F6E00617070656E64546F54DA
:10A4600068696E674465736372697074696F6E00C2
:10A47000617070656E64546F5468696E6750726F76
:10A480007065727479001A1B1C03040607090A1709
:10A4900018191A1B1C03040607090A1718196469FE
:10A4A00073706C6179006C696768744C6576656C73
:10A4B000006D62446973706C6179006D6244697308
:10A4C000706C61794F6666006D62506C6F74006DE0
:10A4D00062556E706C6F74006D6244726177536880
:10A4E000617065006D625368617065466F724C659E
:10A4F00074746572006E656F506978656C53656E33
:10A5000064006E656F506978656C53657450696E50
:10A510000000000000000000010000000200000038
:10A520000300000004000000050000000600000019
:10A530000700000008000000090000000A000000F9
:10A540000B0000000C0000000D0000000E000000D9
:10A550000F000000100000001200000014000000B6
:10A5600016000000180000001A0000001C00000087
:10A570001E00000020000000230000002600000054
:10A58000290000002C0000002F0000003200000015
:10A59000360000003A0000003E00000042000000CB
:10A5A000460000004B000000500000005500000075
:10A5B0005A00000061000000680000006F00000009
:10A5C000760000007D000000840000008B00000089
:10A5D0009200000099000000A0000000A700000009
:10A5E000AE000000B5000000BC000000C300000089
:10A5F000CA000000D1000000D8000000DF00000009
:10A60000E6000000ED000000F4000000FB00000088
:10A61000FF000000000000000008080800080A4AC7
:10A620004000000A5FEA5FEA0ED92ED36E19324469
:10A6300089330C924C924D080800000004880808E9
:10A64000040804848488000A448A4000048EC4807C
:10A65000000000048800000EC00000000008000197
:10A66000224488100C9252524C048C84848E1C829A
:10A670004C901E1EC244924C06CA525FE21FF01E4E
:10A68000C13E02448ED12E1FE24488100ED12ED13D
:10A690002E0ED12EC4880008000800000480048813
:10A6A0000244880482000EC00EC008048244880E52
:10A6B000D126C0040ED135B36C0C925ED2521C92DE
:10A6C0005C925C0ED010100E1C9252525C1ED01C7C
:10A6D000901E1ED01C90100ED013712E12525ED2FE
:10A6E000521C8808081C1FE242524C1254981492C3
:10A6F000101010101E113B75B131113935B3710CAA
:10A700009252524C1C925C90100C92524C861C92AD
:10A710005C92510ED00C825C1FE4848484125252ED
:10A72000524C1131312A44113135BB7112524C92C5
:10A7300052112A4484841EC488101E0EC808080EB4
:10A7400010080482410EC242424E048A40000000BA
:10A750000000001F0804800000000ED2524F1010AD
:10A760001C925C000ED0100E02424ED24E0C925C37
:10A77000900E06C81C88080ED24EC24C10101C92B7
:10A78000520800080808024002424C101498149223
:10A790000808080806001B75B131001C92525200CF
:10A7A0000C92524C001C925C90000ED24EC2000ED5
:10A7B000D010100006C8049808080EC807001252EE
:10A7C000524F0011312A4400113135BB00124C8C1C
:10A7D0009200112A4498001EC4881E06C48C8486E8
:10A7E000080808080818080C881800000C83602561
:10A7F000642025642025642025640A00436F6D7061
:10A80000616374656420466C61736820636F64657E
:10A810002073746F72650A256420627974657320F1
:10A820007573656420282564252529206F662025F9
:10A830006400256420256420256420282564207771
:10A840006F72647329002564207265636F7264738C
:10A850002C20256420776F7264732C206D617849F9
:10A86000442025642C20636F6D70616374696F6E82
:10A87000206379636C6573202564004261642072F3
:10A8800065636F726420666F756E642064757269AB
:10A890006E6720696E697469616C697A6174696F49
:10A8A0006E210A004E6F7420656E6F7567682072A6
:10A8B0006F6F6D206576656E2061667465722063CA
:10A8C0006F6D70616374696F6E0A00526573746FA7
:10A8D0007265642025642073637269707473005319
:10A8E0007461727465640053637269707473206379
:10A8F0006C6561726564002D2D2D2D2D0A0050654B
:10A900007273697374656E74204D656D6F72792012
:10A91000546573740A0A000A496E697469616C6946
:10A920007A696E67204D656D6F72790A004D656DAD
:10A930006F727920696E74697469616C697A656493
:10A940003B2077726974696E67207265636F726409
:10A95000732E2E2E0A005265636F7264206174207C
:10A960006F66667365742025643A2025642025642B
:10A970002025642025642028256420776F72647365
:10A98000290A0046696E616C3A2063757272656EC1
:10A99000742025642075736564202564206330204D
:10A9A00025642063312025640A00E2ECF0F4F8FC11
:10A9B00000046E756D626572006E6F6E65006F7477
:10A9C000686572007061697200737472696E670005
:10A9D000726164696F0064697361626C655261647D
:10A9E000696F006D6573736167655265636569764C
:10A9F0006564007061636B65745265636569766553
:10AA0000007061636B657453656E640072656365A5
:10AA100069766564496E7465676572007265636521
:10AA2000697665644D657373616765547970650017
:10AA30007265636569766564537472696E670073E5
:10AA4000656E64496E74656765720073656E645007
:10AA50006169720073656E64537472696E67007326
:10AA600065744368616E6E656C0073657447726FE0
:10AA7000757000736574506F776572007369676EE7
:10AA8000616C537472656E677468004E6F206672F5
:10AA90006565207461736B20656E747269657300FF
:10AAA0004D656D6F727920636C65617265640041FC
:10AAB0006C6C207461736B732073746F7070656459
:10AAC0000076303633002025732025730073656EC1
:10AAD000736F72730074656D706572617475726501
:10AAE0000074696C74580074696C74590074696CF2
:10AAF000745A00746F7563685265616400693263EB
:10AB000052656164006932635772697465007466E6
:10AB10007400656E61626C65446973706C61790084
:10AB2000736574506978656C006C696E6500726558
:10AB3000637400726F756E6465645265637400635C
:10AB40006972636C6500747269616E676C6500742C
:10AB500065787400746674546F7563686564007416
:10AB60006674546F7563685800746674546F7563C7
:10AB7000685900746674546F7563685072657373B6
:10AB80007572650057656C636F6D6520746F204D3D
:10AB90006963726F426C6F636B732100535049435A
:10ABA0006C6173733A3A535049436C617373284E26
:10ABB00052465F5350495F547970652A2C2075695D
:10ABC0006E74385F742C2075696E74385F742C2035
:10ABD00075696E74385F742900705F737069202125
:10ABE0003D204E554C4C002F55736572732F6A6F84
:10ABF000686E6D616C6F6E65792F4C6962726172FF
:10AC0000792F41726475696E6F31352F7061636B96
:10AC1000616765732F73616E646565706D697374C8
:10AC200072792F68617264776172652F6E52463552
:10AC30002F302E362E302F6C696272617269657307
:10AC40002F5350492F5350492E637070000000005D
:10AC500000000000000000007B4D0000414D00009E
:10AC6000674D0000714D0000A14D0000654D0000D2
:10AC700003000000020000000100000004000000CA
:10AC800005000000110000000C0000000B00000097
:10AC9000120000000A000000060000001A00000078
:10ACA000140000001700000016000000150000004E
:10ACB00010000000FFFFFFFFFFFFFFFF000000008C
:10ACC0001E0000001900000018000000070000002E
:10ACD00008000000090000000D0000000E00000048
:10ACE0000F0000001C0000001B0000001D00000001
:10ACF00013000000000000000000000000003043CE
:10AD000000000000000030C3FB21F93FFB21094097
:10AD10007CD91240FB2119407A6A1F407CD922401D
:10AD2000BBFD2540FB2129403A462C407A6A2F4042
:10AD30005C4731407CD932409C6B3440BBFD354090
:10AD4000DB8F3740FB2139401BB43A403A463C4048
:10AD50005AD83D407A6A3F404C7E40405C47414073
:10AD60006C1042407CD942408CA243409C6B4440D2
:10AD7000AC344540BBFD4540CBC64640DB8F474029
:10AD8000EB584840FB21494083F9A200444E6E0035
:10AD9000FC291500D1572700DD34F50062DBC00027
:10ADA0003C999500419043006351FE00BBDEAB002F
:10ADB000B761C5003A6E2400D24D42004906E0005A
:10ADC00009EA2E001C92D100EB1DFE0029B11C00E7
:10ADD000E83EA700F535820044BB2E009CE98400C4
:10ADE000B4267000417E5F00D6913900538339004C
:10ADF0009CF439008B5F840028F9BD00F81F3B00EC
:10AE0000DEFF97000F980500112FEF000A5A8B0004
:10AE10006D1F6D00CF7E360009CB2700464FB7006F
:10AE20009E663F002DEA5F00BA277500E5EBC7007C
:10AE30003D7BF100F739070092528A00FB6BEA0074
:10AE40001FB15F00085D8D00300356007BFC46009B
:10AE5000F0AB6B0020BCCF0036F49A00E3A91D00D4
:10AE60005E619100081BE60085996500A0145F00F3
:10AE70008D40680080D8FF0027734D000606310022
:10AE8000CA561500C9A873007BE260006B8CC00035
:10AE900002000000030000000400000006000000A3
:10AEA00000000040FB21F93F000000002D44743EEB
:10AEB000000000809846F83C0000006051CC783BD0
:10AEC00000000080831BF0390000004020257A3804
:10AED000000000802282E336000000001DF3693587
:10AEE00000000000000000007D6600006D640000AE
:10AEF000ED66000001670000F7660000796600005B
:10AF00006D6600000D67000099660000696600002C
:10AF1000C872000026720000267200002472000031
:10AF2000BA720000BA720000B07200002472000011
:10AF3000BA720000B0720000BA7200002472000001
:10AF4000C0720000C0720000C07200004A730000AE
:10AF5000C87E0000887D0000887D0000867D00009E
:10AF6000A07E0000A07E0000927E0000867D000092
:10AF7000A07E0000927E0000A07E0000867D000082
:10AF8000A87E0000A87E0000A87E0000A880000027
:10AF90002C2066756E6374696F6E3A20006173735E
:10AFA000657274696F6E2022257322206661696C58
:10AFB00065643A2066696C6520222573222C206C1A
:10AFC000696E65202564257325730A00430000001F
:10AFD0002C020020232D302B2000686C4C0065666D
:10AFE00067454647003031323334353637383941DA
:10AFF00042434445460030313233343536373839F0
:10B0000061626364656600002020202020202020EB
:10B010002028282828282020202020202020202008
:10B020002020202020202020881010101010101028
:10B030001010101010101010040404040404040470
:10B040000404101010101010104141414141410101
:10B0500001010101010101010101010101010101E0
:10B0600001010110101010101042424242424202EF
:10B0700002020202020202020202020202020202B0
:10B08000020202101010102000000000000000005A
:10B0900000000000000000000000000000000000B0
:10B0A00000000000000000000000000000000000A0
:10B0B0000000000000000000000000000000000090
:10B0C0000000000000000000000000000000000080
:10B0D0000000000000000000000000000000000070
:10B0E0000000000000000000000000000000000060
:10B0F0000000000000000000000000000000000050
:10B10000000000000000000000000000000000003F
:10B11000000000000000000000000000000000002F
:10B12000000000000000000000000000000000001F
:10B13000000000000000000000000000000000000F
:10B1400000000000000000000000000000000000FF
:10B1500000000000000000000000000000000000EF
:0CB16000000000000000000000000000E3
:08B16C000850FF7F0100000004
:10B17400FFFFFFFF40060000FEA20000D91F0000F1
:10B1840006A30000D51F00000FA30000DD1F000070
:10B1940018A30000E11F0000EDA30000212400001B
:10B1A400F6A3000075240000FEA300005125000052
:10B1B40006A400008125000010A4000095250000CD
:10B1C40019A400009F25000024A400008B25000082
:10B1D40030A400005F25000041A400007525000094
:10B1E40057A400006925000070A400005525000044
:10B1F400A6A40000C5250000B1A40000792A00001F
:10B20400BBA400000D280000C8A400002D280000E5
:10B21400CFA400007D280000D8A40000CD280000A1
:10B22400E4A40000A52A0000F5A40000B52900004C
:10B2340002A500009526000018000000D6A9000011
:10B24400F5340000E3A900000D380000F3A9000064
:10B25400AD37000001AA0000993900000CAA0000D3
:10B26400113500001CAA00007935000030AA000046
:10B27400213500003FAA0000B33A00004BAA0000A9
:10B284003D3A000054AA0000E33900005FAA000020
:10B29400293700006AAA0000B136000073AA000032
:10B2A400E53600007CAA00002935000019FCFFFFE8
:10B2B400FFFFFFFFFF000000D5AA00003547000094
:10B2C400E1AA0000A14A0000E7AA0000B14A000078
:10B2D400EDAA0000C14A0000F3AA0000694700007B
:10B2E400FDAA0000D14A000005AB0000A9480000F7
:10B2F40012AB00005D4B000020AB0000614B00006E
:10B3040029AB0000654B00002EAB0000694B000028
:10B3140033AB00006D4B00003FAB0000714B0000ED
:10B3240046AB0000754B00004FAB0000794B0000AA
:10B3340054AB00007D4B00005FAB0000814B00006C
:10B3440069AB0000594B000073AB0000554B000083
:10B354000300000002000000080000000A000000D2
:10B36400FFFFFFFF000000000100000000000200DA
:10B3740001000000FFFFFFFF0000000002000000CA
:10B384000000040002000000FFFFFFFF00000000B7
:10B39400030000000000080003000000000000009B
:10B3A40008B1000028B1000048B10000000000000E
:10B3B400000000000000000000000000CCAF00000E
:10B3C4000000000000000000000000000000000079
:10B3D4000000000000000000000000000000000069
:10B3E4000000000000000000000000000000000059
:10B3F4000000000000000000000000002C020020FB
:10B4040007B0000039010000114D00003150000068
:0CB41400716900000D0100000000000044
:040000030000653D57
:00000001FF
